S02000006F70656E626C745F6F6C696D65785F73746D3332653430372E737265630B
S3150800000000000220F9880008498900084989000883
S315080000104989000849890008498900080000000044
S3150800002000000000000000000000000049890008E8
S315080000304989000800000000498900084989000824
S31508000040498900084989000849890008498900083A
S31508000050498900084989000849890008498900082A
S31508000060498900084989000849890008498900081A
S31508000070498900084989000849890008498900080A
S3150800008049890008498900084989000849890008FA
S3150800009049890008498900084989000849890008EA
S315080000A049890008498900084989000849890008DA
S315080000B049890008498900084989000849890008CA
S315080000C049890008498900084989000849890008BA
S315080000D049890008498900084989000849890008AA
S315080000E0498900084989000849890008498900089A
S315080000F0498900084989000849890008498900088A
S3150800010049890008E3620008498900084989000806
S315080001104989000849890008498900084989000869
S31508000120498900084989000849890008E5620008E4
S315080001304989000849890008498900084989000849
S315080001404989000849890008498900084989000839
S315080001504989000849890008498900084989000829
S315080001604989000849890008498900084989000819
S315080001704989000849890008498900084989000809
S30D080001804989000849890008B5
S3150800018810B5054C237833B9044B13B10448AFF3BB
S3150800019800800123237010BD000300200000000022
S315080001A8A48C000808B5034B1BB103490348AFF3F1
S315080001B8008008BD0000000004030020A48C000885
S315080001C872B6704762B67047F0B5002401E001348C
S315080001D8E4B2112C20D8114D15F8147005EB440516
S315080001E895F801E007EB0E0505FB00054AF2104CE9
S315080001F89CFBF5F605FB16C6002EE8D19CFBF5F523
S31508000208ADB20D80013DADB2B5F5806FDFD217707E
S3150800021883F800E00120F0BD0020F0BDE48C00085A
S3150800022810B582B001AB0DF105020DF106014FF4C8
S31508000238FA70FFF7C9FF012804D040F207115048A1
S3150800024800F040FE4F4B00225A611A6842F40042F9
S315080002581A6000F091FB00F1FA044A4B1B6813F484
S31508000268004F05D000F033FF00F086FB8442F4D235
S31508000278444B1A6822F002021A601A6842F0010210
S315080002881A6000F079FB00F1FA043E4B5B6813F03C
S31508000298010F05D100F01BFF00F06EFB8442F4D273
S315080002A89DF805305A1E9DF80430013B1B0543EAA4
S315080002B80243BDF80620013A1343324AD36113684C
S315080002C823F00103136000F057FB00F1FA042D4BE5
S315080002D85B6813F0010F05D000F0F9FE00F04CFB3F
S315080002E88442F4D2284BD3F8002242F00102C3F81C
S315080002F80022D3F8002222F47C52C3F80022D3F84D
S31508000308002242F46062C3F80022D3F8002242F0C1
S315080003180102C3F80022D3F81C2222F48042C3F84B
S315080003281C22D3F80C2242F48042C3F80C22D3F8D4
S31508000338042222F48042C3F80422144AC3F8B022DD
S3150800034802F14C520432C3F8B422D3F8042222F438
S315080003588042C3F80422D3F8142222F48042C3F850
S315080003681422D3F81C2242F48042C3F81C22D3F87C
S31508000378002222F00102C3F8002202B010BD00BF15
S31508000388BC8C000800680040006400400000E0CC0F
S3150800039838B504460D46254B9B6813F0806F3ED04A
S315080003A8224BD3F8802102F00102C3F88021D3F842
S315080003B8802142F07C4242F40012C3F88021C3F837
S315080003C88451E178A278120442EA0162617842EA25
S315080003D8012221780A43C3F88821E179A27912040F
S315080003E842EA0162617942EA012221790A43C3F89D
S315080003F88C21D3F8802142F00102C3F8802100F04D
S31508000408BBFA00F13204094B9B6813F0806F05D1DB
S3150800041800F05DFE00F0B0FA8442F4D238BD40F22E
S315080004288B11034800F04EFDBAE700BF006800408C
S31508000438BC8C0008244BDB6813F0030F41D0224B11
S31508000448D3F8B03113F0040F0ED11F4BD3F8B031DF
S315080004585B0D40F2676293420DD000201A4AD368B2
S3150800046843F02003D3607047174BD3F8B031DB0845
S3150800047843F00043EDE7144BD3F8B42102F00F021A
S315080004880A70D3F8B8210270D3F8B821120A427054
S31508000498D3F8B821120C8270D3F8B821120EC2709C
S315080004A8D3F8BC210271D3F8BC21120A4271D3F8D9
S315080004B8BC21120C8271D3F8BC311B0EC371012002
S315080004C8CCE70020704700BF0068004008B5FFF772
S315080004D877FE08BD10B500F013FA00B910BD04F090
S315080004E8EBFB0028FAD000F0A3FD00F01DFA00F097
S315080004F80BFA20F0604020F07F00044B186000F0EB
S3150800050803FA4468FFF75EFEA047E7E708ED00E050
S3150800051870B508E0461C4D1C0B78037000F0D7FD33
S31508000528304629462246531E9CB2002AF2D170BD8F
S3150800053838B50546002401E00134E4B2082C15D87C
S3150800054800F0C5FD04EB44029300094AD358AB42B0
S31508000558F2D804EB44029100054A0A445268134447
S315080005689D42E9D2024B0B44187A38BDFF2038BDA4
S31508000578088D000808B5C1F3080353B903689942FA
S3150800058809D040F8041B4FF40072FFF7C1FF012099
S3150800059808BD002008BD012008BD2DE9F041074621
S315080005A80068FFF7C5FFFF282DD005F0D5FFF32013
S315080005B805F0EAFF05F0EEFF012816D000247F2C87
S315080005C817D83E68A30006EB03083B445D6800F0AD
S315080005D87EFD2946404606F04DF808280BD156F800
S315080005E824309D420DD10134E9E705F0C5FF002402
S315080005F804E0012400E0002405F0BEFF2046BDE81B
S31508000608F0810024F8E70024F8E7000038B50D461D
S315080006180B4B984208D004460A4B994206D0FFF776
S31508000628BCFF20B9002407E0074C00E0044C294623
S315080006382046FFF79FFF08B1204638BD0024FBE790
S315080006482005002000C000081C0300202DE9F04101
S3150800065806460C4617461D4621F4FF7828F0010879
S315080006680368B3F1FF3F0DD03368984505D0414676
S315080006783046FFF7CBFF064628B33368E41A3444F6
S3150800068804340CE04146FFF775FF03460028EBD112
S3150800069816E017F8013B04F8013B013D0FD000F0BE
S315080006A816FD331DE31AB3F5007FF2D308F500717A
S315080006B83046FFF7ABFF064638B1041DE9E70123C4
S315080006C81846BDE8F0810023FAE70023F8E700009A
S315080006D888422CD838B504460D46022829D90B294C
S315080006E801D9002038BD05F037FFF32005F04CFF87
S315080006F805F050FF01280ED0AC4214D800F0E7FCEC
S3150800070802210D4B33F8140005F07CFF082806D1A2
S315080007180134E4B2F0E705F02FFF002038BD05F0F4
S315080007282BFF002038BD05F027FF012038BD002023
S315080007387047002038BD00BF748D00084FF0FF339E
S31508000748024A1360024A1360704700BF1C03002060
S315080007582005002070B54B1E154C241AA34201D952
S31508000768002070BD16460D460446FFF7E1FEFF2831
S315080007781AD028190138FFF7DBFEFF2816D024F40B
S31508000788FF7323F001030B4A934206D02B463246E1
S3150800079821460948FFF75AFF70BD2B4632462146BF
S315080007A80648FFF753FF70BD002070BD002070BDD6
S315080007B8FFFF0F0800C000081C03002020050020C2
S315080007C84A1E0E4B1B1A9A4201D90020704770B56B
S315080007D80C460546FFF7ACFE064660190138FFF7D2
S315080007E8A7FEFF2E06D0FF2806D001463046FFF79B
S315080007F86FFF70BD002070BD002070BDFFFF0F0899
S31508000808104B1B68B3F1FF3F1AD000B583B00D4AE9
S31508000818536891680B44D1680B4411690B445169B4
S315080008280B4491690B44D26913445B4202AA42F805
S31508000838043D04210448FFF78DFF03B05DF804FB67
S31508000848012070472005002088C100080D4B1B6849
S315080008580D4A126813440D4A126813440C4A126862
S3150800086813440C4A126813440B4A126813440B4A79
S31508000878126813440A4A1268D34201D00020704706
S315080008880120704700C0000804C0000808C0000816
S315080008980CC0000810C0000814C0000818C00008DA
S315080008A888C1000808B50C4B1B68B3F1FF3F04D094
S315080008B80948FFF772FE034650B1084B1B68B3F1A7
S315080008C8FF3F07D00548FFF768FE034600B1012336
S315080008D8184608BD0123FBE7200500201C03002055
S315080008E80048704700C0000808B5FFF727FF08BD8D
S315080008F808B5FFF72FFF08BD08B5FFF761FF08BD64
S3150800090808B5FFF7A3FF08BD08B5FFF7E9FF08BD57
S3150800091808B5FFF775FF034608B9184608BDFFF777
S31508000928C1FF0346F9E700000022014B1A60704729
S3150800093810E000E008B5FFF7F7FF054B054A5A60CF
S3150800094800229A6005211960034B1A6008BD00BF8A
S3150800095810E000E03F90020024070020044B1B68C3
S3150800096813F4803F03D0034A1368013313607047B2
S3150800097810E000E02407002008B5FFF7EFFF014B59
S31508000988186808BD2407002010B5044680210E48BB
S3150800099806F0C0F808B9002010BD21460A4806F036
S315080009A8B1F8FFF7E9FF00F10A048021064806F0C6
S315080009B8B1F838B900F08BFBFFF7DEFF8442F4D2B2
S315080009C8002010BD012010BD0014014010B50446D2
S315080009D82021064806F09EF8012801D0002010BDFF
S315080009E8024806F093F82070012010BD0014014053
S315080009F810B584B04FF4614300930023ADF8043072
S31508000A08ADF80630ADF80830ADF80C300C23ADF863
S31508000A180A30054C6946204605F0FEFF01212046A6
S31508000A2806F062F804B010BD0014014070B5064619
S31508000A380D4640290AD82846FFF7A6FF012803D0FD
S31508000A487D210E4800F03EFA002406E079210B487D
S31508000A5800F038FAEFE70134A4B2ABB29C420BD2E5
S31508000A6800F035FB305DFFF78FFF0128F3D08621AC
S31508000A78024800F027FAEEE770BD00BFA48D00080B
S31508000A8870B5254B1C78BCB92448FFF79FFF012889
S31508000A9801D0204670BD214B1B78013BDBB23F2BAA
S31508000AA8F7D8FFF769FF1E4B186000221D4B1A700E
S31508000AB80122194B1A70ECE706460D46194B1B78A6
S31508000AC8013316481844FFF781FF044601280AD05F
S31508000AD8FFF752FF124B1B686433984219D9002452
S31508000AE80D4B1C70D5E70F4B1A780132D2B21A7023
S31508000AF80A4B1B789A4201D00024CAE70A493046AD
S31508000B08FFF706FD0022044B1A70064B1B782B705C
S31508000B18BFE70024BDE700BF6907002028070020B3
S31508000B286C0700206A07002029070020094B03F1F3
S31508000B381801002232B19A7400225A61054A064BF6
S31508000B481A6070479A745961183318310132D2B24B
S31508000B58F0E700BFA40D0020D40D00200A4B1B683F
S31508000B6883B110B45C69084A146019749860D8602F
S31508000B7800225A741860013908445860987C5DF850
S31508000B88044B7047FF207047D40D002038B504463B
S31508000B980D46012804D940F29D11124800F092F931
S31508000BA862002244D100104B0B445A7C1B7C9A42A3
S31508000BB813D00D4B0B44DA6815705A7C01325A74F7
S31508000BC8DA680132DA605B689A4208D9064A084642
S31508000BD851580244D160012038BD002038BD012093
S31508000BE838BD00BFD08D0008A40D002008B5014601
S31508000BF8024B1878FFF7CAFF08BD00BFD80D0020BA
S31508000C0838B504460D46012804D940F2BF111348E1
S31508000C1800F058F904EB4403DA00114B13445B7CE3
S31508000C28BBB162002244D1000D4B0B449A68127876
S31508000C382A705A7C013A5A749A6801329A605B6833
S31508000C489A4208D9064A0846515802449160012032
S31508000C5838BD002038BD012038BD00BFD08D00083A
S31508000C68A40D002008B50146024B1878FFF7C8FFFF
S31508000C7808BD00BF1C0E002010B50446012804D97B
S31508000C8840F2DF11044800F01DF904EB4404E200C1
S31508000C98024B1344587C10BDD08D0008A40D0020C3
S31508000CA830B583B0FFF742FF0F4C4021601CFFF7B1
S31508000CB855FF20700D4D4021681CFFF74FFF28701F
S31508000CC82378FF2B0BD0FF2809D0094B0093094B33
S31508000CD8094A0121094806F0C1F903B030BD79214E
S31508000CE8074800F0EFF8F0E7D80D00201C0E0020A2
S31508000CF8CC0000204C000020B0000020700700201F
S31508000D08D08D000808B5034807F05BFA002003F001
S31508000D18CFFF08BD7007002070B506460D463F2967
S31508000D280AD82846FFF762FF012803D09E210E48F5
S31508000D3800F0C8F8002406E09A210B4800F0C2F82B
S31508000D48EFE70134A4B2ABB29C420BD200F0BFF96C
S31508000D58305DFFF74BFF0128F3D0A721024800F0C2
S31508000D68B1F8EEE770BD00BFD08D000870B506462D
S31508000D780D461E4807F0CBFC1D4B1C789CB91D4830
S31508000D88FFF770FF012801D0204670BD194B1B7864
S31508000D98013BDBB23E2BF7D80122154B1A7000220D
S31508000DA8154B1A70F0E7144B1B7801331148184491
S31508000DB8FFF758FF0446012801D00024E4E70E4B44
S31508000DC81A780132D2B21A700A4B1B789A4201D0A5
S31508000DD80024D9E709493046FFF79AFB0022044B55
S31508000DE81A70054B1B782B70CEE700BF70070020DA
S31508000DF8A00E0020600E0020A10E0020610E002023
S31508000E0830B583B0144B1878FFF736FF08B3054694
S31508000E18402800D94025002405E09DF807200F4BF7
S31508000E281A550134E4B2A5420DD90DF107010A4B4A
S31508000E381878FFF7E5FE0128EFD040F22711084891
S31508000E4800F040F8E9E72B46044A8121054807F0EF
S31508000E5848F903B030BD00BFD80D0020640D002046
S31508000E68D08D00087007002070B500EB8000C2001E
S31508000E78114B1344B3F88C63002401E00134A4B27F
S31508000E88B4420FD20D4B1D7807F038FE015D28468F
S31508000E98FFF77CFE0128F1D04FF4A371084800F04B
S31508000EA811F8EBE707F02AFE40230246012102481B
S31508000EB807F0E9F870BD00BF700700201C0E002077
S31508000EC8D08D000808B500F002F9FCE708B500F06F
S31508000ED8F9F8012806D000F087F918B10B4B1B78EA
S31508000EE8012B00D008BDFFF747FD094B1B6803F522
S31508000EF81C5310339842F5D30022044B1A7000F09D
S31508000F087DF90028EED1FFF7E5FAEBE7A20E0020F7
S31508000F18A40E002008B50122044B1A70FFF72CFD11
S31508000F28034B1860FFF7D2FF08BD00BFA20E0020CA
S31508000F38A40E002008B5FFF7C9FA00F0C7F8FFF7AE
S31508000F48F9FCFFF7D1FC00F037F900F00FF8FFF7C6
S31508000F58E1FF08BD08B500F0BAF8FFF7FFFC00F096
S31508000F685BFA00F01BF8FFF7B1FF08BD10B503F0F0
S31508000F780DFEFFF755F9084C01232370FFF738FDD6
S31508000F8800232370FFF78CFE0223237000F0CAFCA7
S31508000F980323237010BD00BF0000002000B583B0EE
S31508000FA80DF107012048FFF745FA012817D00DF17A
S31508000FB807011D48FFF764FD012819D00DF107013F
S31508000FC81948FFF7D3FE01281BD00DF1070116486B
S31508000FD800F0FCFC01281DD003B05DF804FB0122D3
S31508000FE8124B1A709DF807100F4803F0EFFDDEE75D
S31508000FF800220E4B1A709DF807100B4803F0E6FD01
S31508001008DCE70222094B1A709DF80710064803F018
S31508001018DDFDDAE70322054B1A709DF8071002482A
S3150800102803F0D4FDD8E700BFA80E00200000002072
S3150800103808B5FFF767FE08BD38B504460D46124BD6
S315080010481B78012B0DD0104B1B7873B10E4B1B78F0
S31508001058022B0FD00C4B1B78032B10D003F0AEFDD8
S3150800106838BDC9B2FFF794F9EDE7E9B22046FFF7AC
S31508001078DDFCEBE7E9B22046FFF74EFEEAE7E9B200
S31508001088204600F085FCE9E700000020054B1B78A0
S31508001098012B05D0022B01D0402070473F2070470E
S315080010A80820704700000020054B1B78012B05D047
S315080010B8022B01D0402070473F2070470820704710
S315080010C80000002008B503F06FFD08BD704770479B
S315080010D810B4034601310D4AA2FB0323DB08F9D1F4
S315080010E800230B70094BA3FB0023DB081A4603EB06
S315080010F883035C00031B303301F8013D1046002AC0
S31508001108F0D108465DF8044B704700BFCDCCCCCC6F
S3150800111800F00F03092802D903F13700704710B504
S3150800112803F1300407F07AFD2044437803F00303FB
S31508001138022B01D0E0B210BD203CFBE738B50546C6
S315080011480C460009FFF7E4FF207005F00F00FFF7CB
S31508001158DFFF60700023A370204638BDF8B5074640
S3150800116800252E4607E0203C10E03301DBB2134485
S31508001178DEB20135EDB2012D19D87C5D07F04EFDBA
S315080011882044437803F00303022BECD0E3B2A3F11F
S315080011983002D2B2162A09D8A3F13A01C9B20629E9
S315080011A807D9092AE1D9373BDAB2DEE700263046FD
S315080011B8F8BD0026FBE7000008B50022064B1A70A2
S315080011C80649074801F056FE00B908BD77210548C3
S315080011D8FFF778FEF9E700BF48130020F88D0008E6
S315080011E8F00E0020FC8D0008034B1B780BB100207D
S315080011F870470120704700BF4813002008B5FFF75D
S3150800120861FF01280ED0084B1B780BB1002008BDDA
S3150800121803F060FD012801D0002008BD0122024B19
S315080012281A7008BD002008BD4813002038B50546C1
S31508001238047807F0F3FC2044437803F00303022BF1
S3150800124803D0532C03D0032038BD203CF9E707F018
S31508001258E5FC6B781844427812F0040F01D1032094
S3150800126838BD312B07D0322B07D0332B01D00320BA
S3150800127838BD022038BD002038BD012038BD70B5FC
S3150800128806460230FFF76AFF054684B2043630463A
S31508001298FFF764FF0544EDB2013CA4B20236012CFF
S315080012A8F5D8ED43EDB23046FFF758FF854201D031
S315080012B8002070BD012070BD2DE9F0410446164690
S315080012C88846A1B198B12046FFF7B0FF054603281E
S315080012D800F099802046FFF7D2FF002800F0978093
S315080012E8012D2DD04DB1022D57D000278CE040F2A4
S315080012F861214848FFF7E6FDE5E7A01CFFF72EFF42
S3150800130887B2201DFFF72AFF0002C8F80000A01DB3
S31508001318FFF724FFD8F800301844C8F80000083446
S31508001328033F3FB2002E6FD0002506E02046FFF7A0
S3150800133815FF705502340135ADB2BD42F6DB63E0E0
S31508001348A01CFFF70BFF87B2201DFFF707FF000455
S31508001358C8F80000A01DFFF701FFD8F8003003EB16
S315080013680020C8F8000004F10800FFF7F7FED8F8CF
S3150800137800301844C8F800000A34043F3FB2002E6B
S3150800138842D0002506E02046FFF7E8FE70550234ED
S315080013980135ADB2BD42F6DB36E0A01CFFF7DEFE2E
S315080013A887B2201DFFF7DAFE0006C8F80000A01D60
S315080013B8FFF7D4FED8F8003003EB0040C8F8000061
S315080013C804F10800FFF7CAFED8F8003003EB00203E
S315080013D8C8F8000004F10A00FFF7C0FED8F8003084
S315080013E81844C8F800000C34053F3FB266B100251A
S315080013F806E02046FFF7B2FE705502340135ADB255
S31508001408BD42F6DB00E000273846BDE8F0814FF01C
S31508001418FF37F9E7FC8D0008964B1B78002B00F080
S31508001428F18170B5012B05D0022B2DD0032B00F0C6
S315080014383F8170BDFFF758FA03F06EFC8E4803F03B
S31508001448AFFC8E4803F0ACFC03F062FC01220146AF
S315080014588B4801F03BFD30B18A4803F0A1FC012016
S3150800146803F090FC70BD884803F09AFC874803F09F
S3150800147897FC874803F094FC864B00221A605A604A
S3150800148802227C4B1A7070BD834C04F50C724FF41B
S315080014988071824802F034F994F84132002B5ED103
S315080014A8002877D07D48002200F5C071FFF704FFB1
S315080014B80446B0F1FF3F60D0002C09DD754B5B6828
S315080014C8002B69D1754BD3F88021724B1A605C6082
S315080014D8714BD3F84422D3F83C329A42A9D1002159
S315080014E8674801F0C9FF002840F0A980694B5B6886
S315080014F873B3654803F054FC694803F051FC694D19
S31508001508644C29466068FFF7E3FD284603F048FC63
S31508001518654803F045FC2946E078FFF70FFEA91C45
S31508001528A078FFF70BFE291D6078FFF707FEA91DAF
S315080015382078FFF703FE284603F032FC5B4803F0E1
S315080015482FFC61682068FFF7D7F9002800F0848027
S315080015584D4803F025FC0322464B1A7070BD4948CE
S3150800156803F01EFC022003F00DFC04F50C7001F0D4
S315080015786FFF00223F4B1A7070BD424803F010FCFB
S31508001588032003F0FFFB3E4801F062FF0022394BB7
S315080015981A7070BD00248FE7404AD2F880113D4A78
S315080015A812681A44914239D0374803F0F9FB3C4887
S315080015B803F0F6FB3B4E374D31466868FFF788FD62
S315080015C8304603F0EDFB384803F0EAFB3146E87885
S315080015D8FFF7B4FDB11CA878FFF7B0FD311D687890
S315080015E8FFF7ACFDB11D2878FFF7A8FD304603F0D4
S315080015F8D7FB2E4803F0D4FB69682868FFF77CF9FF
S3150800160880B1214803F0CCFB214803F0C9FB234BE2
S31508001618D3F880211F4B1A605C6059E723441D4A9A
S31508001628536055E7174803F0BBFB052003F0AAFBF0
S31508001638134801F00DFF00220E4B1A7070BD1148B1
S3150800164803F0AEFB042003F09DFB0D4801F000FFF4
S315080016580022084B1A7070BD0A4803F0A1FB052042
S3150800166803F090FB064801F0F3FE0022014B1A70BE
S3150800167870BD00BF48130020188E00083C8E00086D
S3150800168820110020648E00086C8E0008748E0008ED
S31508001698988E0008E80E0020F00E00204C13002053
S315080016A8C88E0008D0140020D48E0008788F000849
S315080016B8554C04F50C724FF48071544802F020F822
S315080016C894F84132002B66D100287FD04F4800F5A0
S315080016D8807200F5C071FFF7EFFD0546B0F1FF3FD0
S315080016E867D0002D34DD4A4803F05AFB494C214699
S315080016F82846FFF7EDFC204603F052FB464803F060
S315080017084FFB424E214696F88301FFF717FDA11CA9
S3150800171896F88201FFF712FD211D96F88101FFF759
S315080017280DFDA11D96F88001FFF708FD204603F078
S3150800173837FB3A4803F034FB06F580722946D6F893
S315080017488001FFF7D5F8002842D0354803F028FB72
S315080017582D4BD3F84422D3F83C329A427FF469AE2B
S31508001768304803F01DFBFFF7D3F800283DD02C4876
S3150800177803F016FB2C4803F013FB2C4801F068FE0F
S315080017882B4803F00DFB00222A4B1A7003F0D8FAEF
S31508001798FEF7A0FE4DE6284803F002FB022003F0F8
S315080017A8F1FA04F50C7001F053FE0022214B1A7069
S315080017B870BD224803F0F4FA032003F0E3FA1B4845
S315080017C801F046FE00221B4B1A7070BD002588E7FB
S315080017D81B4803F0E5FA062003F0D4FA134801F08B
S315080017E837FE0022134B1A7070BD154803F0D8FA55
S315080017F8072003F0C7FA0D4801F02AFE00220D4B10
S315080018081A7070BD704700BFF00E00204C130020F8
S31508001818388F0008D0140020488F0008788F0008F1
S315080018286C8E0008608F00087C8F00082011002045
S31508001838948F000848130020F08E0008148F0008BB
S31508001848648E000810B505F08FFA98B9FFF794F872
S315080018582E4B1B68984206D303F5FA732B4A136076
S315080018680024002C33D0FFF787F8294B1B689842C9
S3150800187843D210BD274A1080274B9C894FF4006035
S3150800188802F0A4F8844213D0234B9C8940F606003C
S3150800189802F09CF88442D9D102F0EEFE1D4B1B8853
S315080018A8002BD3D005F084FA00221A4B1A80CDE70C
S315080018B8012002F0C5F8174B1B88002BC6D002F08A
S315080018C84DFF05F075FA0022124B1A80BEE7134A37
S315080018D8682303FB0423124A1360022002F0B0F8B7
S315080018E80C4B1B880BB90134BBE702F037FF05F030
S315080018F85FFA0022074B1A80F5E703F51C531033E5
S31508001908034A136002F084FEB3E700BF14150020EB
S3150800191810150020FC1A00208C1B0020141B002020
S31508001928101B002008B505F02BF9FFF725F800F578
S31508001938FA70124B1860FFF71FF800F51C501030A4
S315080019480F4B186001F0FCFF0E4B4FF6A9621A8080
S3150800195843F6137159800C4B4FF6FF711980002115
S3150800196859800A4B1A8040F213125A804EF6030021
S3150800197802F014F805F0E8F908BD00BF14150020B0
S3150800198810150020881B0020841B0020801B0020BF
S3150800199838B50D4B1D68EB692B62002306E01A1D46
S315080019A8C45C2A4482F8204001339BB28AB2934227
S315080019B8F5D3111DA5F8641005F1200002F094FD71
S315080019C8EB690133EB6138BD101B002008B5FFF73A
S315080019D839FF002008BD000010B5184B1C68184BC5
S315080019E81B7813F0400F11D113F0010F02D0002213
S315080019F8A4F8642013F0040F02D0B4F8641059B997
S31508001A080F4B1B7813F0020F0BD110BD0123E361AE
S31508001A180023A4F8643010BD04F1200002F064FD28
S31508001A28EEE70023A4F86430064B1868064B1978C5
S31508001A380439C9B2043003F0C9F8E6E7101B0020D8
S31508001A48081B00200C1B0020FC1A0020427800788E
S31508001A5840EA02207047C278837843EA022243782C
S31508001A6843EA0223007840EA032070470170090A0E
S31508001A78417070470170C1F307234370C1F30743E8
S31508001A888370090EC170704713462AB10A78027026
S31508001A9801300131013BF9D1704701700130013A33
S31508001AA8FBD1704730B4451C037808781B1A013AED
S31508001AB804D04C1C28462146002BF4D0184630BCC6
S31508001AC8704700E0013003780BB18B42FAD118460B
S31508001AD8704702394369023B994204D24389806AAE
S31508001AE803FB010070470020704770B506460D468F
S31508001AF801F11A00FFF7AAFF04463378032B00D032
S31508001B0870BD05F11400FFF7A1FF44EA0040F7E7A6
S31508001B1870B506460C46154691B204F11A00FFF749
S31508001B28A5FF3378032B00D070BD290C04F11400E7
S31508001B38FFF79CFFF8E700002DE9F04180460F46BD
S31508001B4801F11A00FFF782FF58BB3D7805F03F05FB
S31508001B58013D05EB450305EB83050126002404E052
S31508001B684FF6FF73984222D101340C2C0DD8144B2A
S31508001B78185D3844FFF76AFF002EF1D0FE2D13D8FA
S31508001B8828F8150006460135EEE73B7813F0400FAE
S31508001B9810D0FE2D11D8002328F815300120BDE8ED
S31508001BA8F0810020BDE8F0810020BDE8F081002022
S31508001BB8BDE8F0810120BDE8F0810020BDE8F0818C
S31508001BC8409000082DE9F84380460F4691464B7326
S31508001BD80F23CB7200240C73214607F11A00FFF76E
S31508001BE845FF09F1FF3606EB460306EB830625464D
S31508001BF802E001340C2C11D84FF6FF739D4202D02F
S31508001C0838F8165001360C4B185D29463844FFF744
S31508001C182DFF002DEDD14FF6FF75EAE74FF6FF7356
S31508001C289D4202D038F816300BB949F0400987F8B2
S31508001C380090BDE8F88300BF4090000870B582B0F0
S31508001C48054616461C460B22FFF71EFF052C11D81B
S31508001C5807231FE001310F290DD802F0010000EB18
S31508001C684303520813F4803FF4D083F4883383F08F
S31508001C782103EFE72346328812B102360021EAE744
S31508001C881C46E5E75A1E02A8034403F8081C24095B
S31508001C9809D0134604F00F0202F130013929F1D9A7
S31508001CA802F13701EEE77E210346134403F8081CC0
S31508001CB800E00134944208D22B5D202BF9D104E0C8
S31508001CC8202018700C46072909D8611C2B19072AE1
S31508001CD8F6D802A8104410F8080C0132F1E702B049
S31508001CE870BD01460B220020C30143EA5003087859
S31508001CF850FA83F3D8B20131013AF5D17047016831
S31508001D0809B10A4603E04FF0FF3308E001321378B9
S31508001D181F2B01D93A2BF9D13A2B02D000231846A2
S31508001D28704710B44C1C0B78303B092B08D8A242D4
S31508001D3809D15BB90132026018465DF8044B704751
S31508001D484FF0FF33F8E74FF0FF33F5E74FF0FF336F
S31508001D58F2E738B50C4620B1054603680BB11A7880
S31508001D681AB900232360092038BDD9888288914288
S31508001D78F7D1587804F0CCFA10F0010FF1D12B6896
S31508001D882360002038BDF8B5C3780BB90020F8BD24
S31508001D980446C66A00F130070123324639464078B8
S31508001DA804F0F4FAA8B90023E370236AF31AA269BF
S31508001DB8934210D2A57808E0A3691E440123324647
S31508001DC83946607804F0E2FA013D012DF4D800207E
S31508001DD8F8BD0120F8BD0020F8BD70B5C36A8B426E
S31508001DE814D004460D46FFF7CEFF064608B130461E
S31508001DF870BD01232A4604F13001607804F09CFA84
S31508001E0810B101264FF0FF35E562F0E70026EEE748
S31508001E1810B504460023C3704FF0FF33C362FFF7BB
S31508001E28DCFF08B1042010BD04F22E20FFF70EFED1
S31508001E384AF65523984201D0032010BD04F16600DE
S31508001E48FFF709FE20F07F40084B98420CD004F1B2
S31508001E588200FFF700FE20F07F40044B984201D02D
S31508001E68022010BD002010BD002010BD46415400B8
S31508001E782DE9F04784B00E46174600230B60FFF796
S31508001E883EFF051EC0F23581A84B53F82540002CA5
S31508001E9800F03381346007F0FE0723787BB1607859
S31508001EA804F036FA10F0010F09D1002F00F0278147
S31508001EB810F0040F01D00A201CE100201AE10023C3
S31508001EC82370E8B2607004F00BFA10F0010F01D025
S31508001ED803200FE127B110F0040F01D00A2009E109
S31508001EE800212046FFF794FF02281DD00026042863
S31508001EF800F0078101282DD90D20FBE0002004AB4E
S31508001F0803EB850343F8100C0135032D0ED804F1AD
S31508001F1830002B0103F5DF7318440379002BEDD045
S31508001F280830FFF798FDEAE70025EEE7002508E000
S31508001F3831462046FFF76CFF0128D8D90135032D0D
S31508001F48D5D804AB03EB850353F8106C002EEFD1F4
S31508001F580320F1E704F13B00FFF778FDB0F5007FB1
S31508001F6801D00D20C6E004F14600FFF76FFD804654
S31508001F7820B904F15400FFF76EFD8046C4F81880AE
S31508001F8894F8409084F8029009F1FF33DBB2012BEC
S31508001F9801D90D20AEE009FB08F994F83D70678170
S31508001FA8002F00F0B0807B1E1F4201D00D20A1E053
S31508001FB804F14100FFF74AFD8246208110F00F0F11
S31508001FC840F0A38004F14300FFF740FD054620B919
S31508001FD804F15000FFF73FFD054604F13E00FFF700
S31508001FE835FD0246002800F0928009EB000303EB52
S31508001FF81A139D42C0F08D80ED1AB5FBF7F5002D32
S3150800200800F0898040F6F5718D4260D801274FF6B1
S31508002018F5718D4200D9032702356561E6613244B8
S3150800202822623344A362032F53D104F15A00FFF7FF
S315080020380DFD002871D1BAF1000F70D104F15C00CA
S31508002048FFF709FD6062AD0005F2FF15B8EB552FDD
S3150800205869D34FF0FF332361E36080232371032F8D
S315080020682CD104F16000FFF7F1FC012826D1711C78
S315080020782046FFF7B2FE08BB0023237104F22E2080
S31508002088FFF7E4FC4AF65523984217D104F13000C5
S31508002098FFF7E1FC264B984210D104F50570FFF7C7
S315080020A8DAFC244B984209D104F50670FFF7D3FCED
S315080020B8206104F50770FFF7CEFCE06027701E4A1A
S315080020C8138801339BB21380E380002012E00227AD
S315080020D89DE7BAF1000F24D04A446262022F01D163
S315080020E86D00B1E705EB450305F0010505EB53055A
S315080020F8AAE70B2004B0BDE8F0870C20FAE7002011
S31508002108F8E70120F6E70D20F4E70D20F2E70D20A1
S31508002118F0E70D20EEE70D20ECE70D20EAE70D20A5
S31508002128E8E70D20E6E70D20E4E700BF18150020CC
S3150800213852526141727241611C150020F8B5066851
S3150800214801295DD9736999425CD20C463378022B0A
S3150800215830D0032B40D0012B01D00120F8BD01EB6C
S315080021685105316A01EB55213046FFF736FE10B1A5
S315080021784FF0FF30F8BD6F1CC5F30805354495F8D0
S315080021883050316A01EB57213046FFF726FE10B169
S315080021984FF0FF30F8BDC7F308073E4496F83000FD
S315080021A845EA002014F0010F01D00009F8BDC0F374
S315080021B80B00F8BD316A01EB14213046FFF70DFE16
S315080021C810B14FF0FF30F8BD600000F4FF703030F2
S315080021D83044FFF73BFCF8BD316A01EBD4113046B1
S315080021E8FFF7FBFD10B14FF0FF30F8BDA00000F473
S315080021F8FE7030303044FFF72EFC20F07040F8BDF2
S315080022080120F8BD0120F8BD2DE9F0410768B1F5B0
S31508002218001F02D30220BDE8F08106460C4611F0DD
S315080022281F0F02D00220BDE8F081316185681DB90B
S315080022383B78022B00D97D6A75B93B89B3EB541FE5
S3150800224802D80220BDE8F0817B6AB3617561B3697B
S315080022580BBB0220BDE8F081B7F80A804FEA482888
S3150800226801E0A4EB080444450FD329463046FFF796
S3150800227865FF0546B0F1FF3F18D0012819D97B69D3
S315080022889842EED30220BDE8F08129463846FFF782
S3150800229820FCB061DAE703EB5423B3613037C4F3A3
S315080022A808043C44F4610020BDE8F0810120BDE83B
S315080022B8F0810220BDE8F0812DE9F84301297ED98D
S315080022C84369994201D302267AE017460C46054621
S315080022D80378022B47D0032B57D0012B01D00226AF
S315080022E86EE001EB5108016A01EB5821FFF775FD0D
S315080022F80646002864D108F10109C8F3080814F04D
S31508002308010423D005EB080393F9303003F00F03D3
S315080023183A0102F47F621343DBB2A84488F83030E6
S315080023280123EB70296A01EB59212846FFF755FD69
S315080023380646002844D1C9F308094CB1C7F3071261
S31508002348A94489F830200123EB7039E0FBB2E4E7A9
S3150800235805EB090393F9302022F00F02C7F3032788
S315080023683A43D2B2ECE7016A01EB1421FFF735FDCF
S31508002378064628BB600000F4FF703030B9B228441E
S31508002388FFF774FB0123EB701AE0016A01EBD4111D
S31508002398FFF723FD064698B927F07047A40004F40A
S315080023A8FE7430342C442046FFF755FB00F0704184
S315080023B839432046FFF75EFB0123EB7000E002264F
S315080023C83046BDE8F8832DE9F04107460668884691
S315080023D831B9F5688DB173699D420FD301250DE0B2
S315080023E8FFF7ACFE0346012847D9B0F1FF3F49D0AD
S315080023F87269904246D3454600E001252C460CE012
S3150800240821463846FFF79AFE034670B1012839D0A7
S31508002418B0F1FF3F36D0AC4233D0013473699C42E1
S31508002428EED3012D2BD90224EAE74FF0FF322146D5
S315080024383046FFF741FF034610B9B8F1000F0ED131
S31508002448A3B9F46033697269023A934201D2013B2F
S315080024583361337943F001033371234612E0224688
S3150800246841463046FFF728FF0346E9E7012B01D026
S31508002478012307E04FF0FF3304E0012302E00023BD
S3150800248800E000231846BDE8F081F8B50E46046852
S31508002498012930D90746114663699E4201D30222AB
S315080024A82AE05AB14FF0FF322046FFF705FF0246E9
S315080024B820B121E063692E469D421DD23146384631
S315080024C8FFF73CFE0546C8B1012819D0B0F1FF3F11
S315080024D818D0002231462046FFF7EEFE024658B9C4
S315080024E82369B3F1FF3FE5D001332361237943F02C
S315080024F801032371DEE702221046F8BD0022FBE736
S315080025080222F9E70122F7E72DE9F8430668036985
S3150800251803F12005836913B90420BDE8F883B5F5E6
S31508002528001F02D30420BDE8F88388460446C5F38D
S3150800253808078FB901338361416941B93389B3EB18
S31508002548551F09D8002383610420BDE8F8837389D9
S31508002558013B13EA552307D0256107F1300846449D
S31508002568E6610020BDE8F883FFF7E8FD8146012803
S3150800257848D9B0F1FF3F48D0736998423AD3B8F1C1
S31508002588000F04D10023A3610420BDE8F88361691C
S315080025982046FFF718FF814610B90720BDE8F883DB
S315080025A8012835D0B0F1FF3F35D03046FFF7EBFBB1
S315080025B8A0BB4FF40072002106F13000FFF76DFA50
S315080025C849463046FFF785FAF0624FF000087389E6
S315080025D898450BD20123F3703046FFF7D4FB00BBAE
S315080025E808F10108F36A0133F362F0E7F36AA3EB2B
S315080025F80803F362C4F8149049463046FFF769FAA7
S31508002608A061A9E70220BDE8F8830120BDE8F883A0
S315080026180220BDE8F8830120BDE8F8830120BDE85B
S31508002628F8830120BDE8F883F8B504460F4606681E
S315080026380021FFF7E9FD0246C0B9002508E0013583
S31508002648BD4213D001212046FFF75EFF024668B94E
S31508002658A1693046FFF7C1FB024638B9E3691B781A
S31508002668E52BECD0002BEAD00025EBE7042A01D0AD
S315080026781046F8BD0722FBE72DE9F84304468846C5
S3150800268807684FF0FF094E4604252EE00F2B19D18F
S3150800269812F0400F06D091F80D9002F0BF02236998
S315080026A863621646B24201D0FF2618E04B7B99456D
S315080026B801D0FF2613E0A06AFFF73EFA88B3013E69
S315080026C8F6B20CE026B90846FFF70BFB81452BD076
S315080026D84FF0FF33636227E0FF2600E0FF2600215C
S315080026E82046FFF711FF0546F0B9A169E1B138465A
S315080026F8FFF773FB0546B8B9E1690A789AB1CB7A48
S3150800270803F03F03A371E52AE6D02E2AE6D023F084
S315080027182000082814BF002001204045B6D0FF260F
S31508002728DDE7FF26DBE704250DB10023A36128466C
S31508002738BDE8F88370B5044605680669416AB1F1CB
S31508002748FF3F1CD0FFF760FD0346B3B9A1692846C9
S31508002758FFF743FB034670B9E269E52111700122C8
S31508002768EA702269964206D900212046FFF7CCFE70
S3150800277803460028EAD0042B03D0184670BD002368
S31508002788E3E70223F9E700002DE9F04F83B0064690
S315080027988A46D1F80090856A002412E0013709EBC9
S315080027A8070219F807302F2BF8D05C2BF6D0CAF891
S315080027B800201F2822D84FF0040823E025F81480A3
S315080027C83C46671C19F804001F28E8D92F28E6D0C4
S315080027D85C28E4D0FE2C00F2DD80012100F0E2FF3F
S315080027E88046002800F0D8807F28E7D801466B483D
S315080027F8FFF767F90028E1D0062012E04FF0000835
S3150800280800E0013C44B104F10043013B35F81330BC
S31508002818202BF6D02E2BF4D0002325F814301CB91B
S31508002828062003B0BDE8F08F0B222021306AFFF797
S3150800283834F9002300E0013335F81320202AFAD0AA
S315080028482E2AF8D01BB148F0030800E0013C6CB109
S3150800285804F10042013A35F812202E2AF6D14FF033
S31508002868080B4FF0000ACDF804A00AE0A2464FF07C
S31508002878080B0022019204E04C450BD048F00308E7
S315080028884B4603F1010935F8137057B3202FF5D0D5
S315080028982E2FF1D0DA450FD24C450DD07F2F3FD8D1
S315080028A8002F4AD148F003085F27336A03F80A70ED
S315080028B84B460AF1010AE4E7BBF10B0F0FD04C456A
S315080028C801D048F003084C450BD3019B9B00DBB2AB
S315080028D8019323464FF00B0B4FF0080AD1E748F04F
S315080028E80308336A1A78E52A43D0BBF1080F43D0A0
S315080028F8019901F00C020C2A43D001F00303032BBB
S315080029083FD018F0020F06D1019B03F00303012BF1
S315080029183AD0042A3BD0336A83F80B80002080E734
S315080029280021384600F03EFF074618B1A0F1800797
S315080029381B4BDF5D48F00208B2E739461948FFF72E
S31508002948C0F80028AED1A7F141039BB2192B04D8C9
S31508002958019B43F002030193A7E7A7F161039BB222
S31508002968192BA2D8019B43F001030193203FBFB25C
S315080029789BE705221A70B8E7019B9B00DBB2019317
S31508002988B6E748F00208BCE748F01008C1E748F07F
S315080029980808C0E7062044E7062042E750900008E2
S315080029A8C08F00085C900008F8B500238B7583690A
S315080029B8002B6BD00D460646436AB3F1FF3F13D08A
S315080029C8836A00249F1C188858B1002100F0EAFE83
S315080029D830B1FE2C0CD82A1990753B460134F1E71C
S315080029E800242C440023A375AC7D0022134612E06C
S315080029F80024F6E7E52317E014B9A8182E278775E3
S31508002A08A8182E274772013210E010271CE0A818CC
S31508002A18837501320B460A2B1BD8F069591CC35C0F
S31508002A28202BF7D0052BE5D00929E5D0A81843723D
S31508002A38002CEED1A3F14100C0B21928E7D8F069F5
S31508002A48007B0829E1D808270742E0D02033DBB203
S31508002A58DDE734B9AB1800219975F3691B7B03B90F
S31508002A680A462A4400235372F369DB7A2B72F06903
S31508002A781C30FEF7F0FF2860F0691830FEF7E6FF0D
S31508002A88A880F0691630FEF7E1FFE880F8BD000077
S31508002A982DE9F0478146884601F11A00FEF7D6FF68
S31508002AA8B0BB98F8005005F03F05013D05EB450316
S31508002AB805EB83050127002404E04FF6FF739842C7
S31508002AC82FD101340C2C17D81C4B185D4044FEF73F
S31508002AD8BDFF0646002FF0D0FE2D1CD800F07EFE5E
S31508002AE8074605F1010A39F8150000F077FE87420E
S31508002AF814D137465546E4E798F8003013F0400FE6
S31508002B0812D0A7B139F81530A3B90120BDE8F08766
S31508002B180020BDE8F0870020BDE8F0870020BDE862
S31508002B28F0870020BDE8F0870120BDE8F08701207E
S31508002B38BDE8F0870020BDE8F08700BF4090000890
S31508002B482DE9F8430446D0F800800021FFF75CFB1E
S31508002B58064600285ED14FF0FF3363624FF0FF093F
S31508002B684F460AE04FF0FF336362FF2700212046ED
S31508002B78FFF7CAFC064600284CD1A1694046FFF76C
S31508002B882CF90646002845D1E5692B78002B40D054
S31508002B98E97A01F03F02A271E52BE3D011F0080F9C
S31508002BA801D00F2ADED10F2A14D027B92846FFF7F5
S31508002BB898F881452ED0216ACB7A13F0010F04D1F3
S31508002BC80B222846FEF76EFF20B34FF0FF336362E9
S31508002BD8FF27CBE7A06A0028C8D013F0400F06D015
S31508002BE895F80D9003F0BF03226962621F46BB423F
S31508002BF801D0FF27BAE76B7B994501D0FF27B5E7D0
S31508002C082946FFF745FF10B1013FFFB2AEE7FF2798
S31508002C18ACE704263046BDE8F88330B583B00446E9
S31508002C280191056801E001330193019B1A782F2A5F
S31508002C38F9D05C2AF7D00022A2601B781F2B1DD971
S31508002C4801A92046FFF7A0FD0346F8B92046FFF775
S31508002C5877FF236ADA7A0346D8B912F0040F15D132
S31508002C68A37913F0100F1BD02169C1F3080130317D
S31508002C7829442846FEF739FFA060E1E7236A80223F
S31508002C88DA7200212046FFF7BFFA0346184603B052
S31508002C9830BD0428FAD112F0040FF7D10523F5E759
S31508002CA80523F3E72DE9F04784B00668D0F820A095
S31508002CB8D0F828809AF80B3013F0A00F05D04FF0FB
S31508002CC80609484604B0BDE8F087002400E0013448
S31508002CD838F81430002BFAD105460C22514601A8BB
S31508002CE8FEF7D2FE9DF80F3013F0010F1ED0002311
S31508002CF88AF80B30AB620127632F0CD83B4642464D
S31508002D0801A95046FEF79AFF2846FFF719FF81469C
S31508002D1808B90137F0E7642F60D0B9F1040FD0D1AC
S31508002D289DF80F308AF80B30C5F828809DF80F30C3
S31508002D3813F0020F2AD00C342A4BA3FB0434A40838
S31508002D48013421462846FFF76FFC814608B9013C3D
S31508002D581ED1B9F1000FB4D1A9693046FFF73DF87D
S31508002D6881460028ADD120220021E869FEF795FEA4
S31508002D780B22296AE869FEF787FEEA692B6ADB7A75
S31508002D8803F0180313730123F3709AE70124D8E7AD
S31508002D982969A1EB44112846FFF736FA8146002827
S31508002DA8D7D1286AFEF79DFF0746A9693046FFF777
S31508002DB814F881460028CCD13B46E2B2E969A86AEC
S31508002DC8FEF700FF0123F37000212846FFF79CFB56
S31508002DD881460028BDD1013CE7D1BAE74FF007097B
S31508002DE86FE700BF4FECC44E70B50446FEF7CBFF3D
S31508002DF8054648B92378032B08D00022114660787F
S31508002E0803F0F0FA00B10125284670BD2379012B95
S31508002E18F3D104F130064FF4007200213046FEF76C
S31508002E283CFE4AF6552104F22E20FEF71FFE0F49EE
S31508002E383046FEF71FFE0E4904F50570FEF71AFE22
S31508002E48216904F50670FEF715FEE16804F50770B2
S31508002E58FEF710FEE2690132E26201233146607824
S31508002E6803F094FA00232371C7E700BF5252614161
S31508002E787272416110B584B001900091144604A895
S31508002E8840F8041DFEF73BFF002818DB0E4B53F8E5
S31508002E9820300BB100221A70019B0BB100221A7060
S31508002EA8019B094A42F8203063B1012C01D0002061
S31508002EB806E0002201A96846FEF7DAFF00E00B20C3
S31508002EC804B010BD0020FBE7181500202DE9F043D3
S31508002ED893B00191002800F0AE80044616460023F8
S31508002EE8036002F01F073A4606A901A8FEF7C0FFC5
S31508002EF80546002840F0A080069B079303AB0F936E
S31508002F084F4B1193019907A8FFF787FE054620B985
S31508002F180F9B93F90B30002B2FDB16F01C0F79D07B
S31508002F28002D31D0042D2AD047F0080715B917F017
S31508002F38080F35D14DB917F0080F01D047F020070B
S31508002F48069BDB6A23620E9B6362002D74D1069E7C
S31508002F58DDF8388041463046FEF7C7FDA06008F11F
S31508002F681C00FEF778FDE060002363746361E36183
S31508002F7827742660F388A3805EE00625CDE707A8B0
S31508002F88FFF790FE0546CFE79DF8223013F0110F9C
S31508002F9804D116F0040FC9D00825C7E70725C5E7E1
S31508002FA8284E31460E980E30FEF764FD31460E98C7
S31508002FB81630FEF75FFD20220E9BDA72069EDDF8B4
S31508002FC8388041463046FEF790FD81460022414644
S31508002FD83046FEF79DFD00210E981C30FEF74AFD87
S31508002FE80122069BDA70B9F1000FA3D0069BDE6AA8
S31508002FF80022494607A8FFF748FA0546002899D146
S3150800300831460698FEF7E9FE054609F1FF33069AA2
S31508003018D3608FE7002D8DD19DF8223013F0100F5D
S3150800302807D116F0020F85D013F0010F82D00725B5
S3150800303880E704257EE70925284613B0BDE8F0830E
S3150800304820150020000061482DE9F04F85B0044698
S315080030588846164699460023C9F8003003A9FEF79C
S3150800306878FE074630B9677C27B9237C13F0010F29
S3150800307804D10727384605B0BDE8F08FE3686269CA
S315080030889B1AB34253D21E4651E0A1692046FFF760
S3150800309855F85EE002276774ECE701276774E9E7E5
S315080030A802276774E6E701276774E3E74FF40072B7
S315080030B804F1280108EB4020FEF7E6FC74E0E26913
S315080030C8019B934219D0237C13F0400F0BD00123A0
S315080030D804F12801687803F059F9002867D1237C98
S315080030E823F0400323740123019A04F12801039865
S315080030F8407803F021F900285CD1019BE3616169F6
S31508003108C1F30801C1F50075AE4200D2354628312B
S315080031182A4621444046FEF7B7FCA84463692B446F
S315080031286361D9F800302B44C9F80030761B002EA5
S31508003138A0D06369C3F30802002AE0D1039AB2F85B
S315080031480AA00AF1FF3A1AEA532A08D1002B9CD199
S31508003158A06801289ED9B0F1FF3F9ED0A061039DC3
S31508003168A1692846FEF7B5FC002899D00AEB0003A2
S3150800317801935FEA562BA2D00AEB0B036A8993429E
S3150800318801D9A2EB0A0B5B46019A4146687803F017
S31508003198D3F8002887D1237C13F0400F04D0E069C0
S315080031A8019BC01A834581D84FEA4B25B5E7012705
S315080031B867745FE7012767745CE72DE9F04F85B008
S315080031C804468846164699460023C9F8003003A9D6
S315080031D8FEF7BFFD074630B9677C27B9237C13F08D
S315080031E8020F04D10727384605B0BDE8F08F636992
S315080031F8F3425FD3DE435DE000212046FFF7E3F89C
S315080032086CE0A1692046FFF7DEF867E002276774D5
S31508003218E9E701276774E6E70123E26904F128016B
S315080032280398407803F0B2F820B9237C23F04003CA
S31508003238237462E001276774D5E702276774D2E723
S3150800324801276774CFE74FF4007208EB412104F1B0
S315080032582800FEF719FC237C23F0400323746EE04C
S31508003268E3699B4503D06269E3689A4269D3C4F85F
S315080032781CB06069C0F30800C0F50075AE4200D2FC
S31508003288354628302A4641462044FEF7FDFB237C6E
S3150800329843F040032374A84463692B446361E268D6
S315080032A8934238BF1346E360D9F800302B44C9F86F
S315080032B80030761B002E51D06369C3F30802002A32
S315080032C8D7D1039AB2F80AA00AF1FF3A1AEA532A9A
S315080032D80FD1002B95D1A06800288DD000283DD0A5
S315080032E8012893D0B0F1FF3F93D0A061A36803B932
S315080032F8A060237C13F0400F8ED1039B0193A1692C
S315080033081846FEF7E6FB8346002896D0D344750A86
S31508003318A6D00AEB0503019A5289934201D9A2EB72
S315080033280A052B465A4641460198407803F02EF876
S31508003338002885D1E169A1EB0B018D4283D86D027E
S31508003348A9E701235A4604F128010198407802F0B2
S31508003358F3FF00288BD00127677444E7237C43F0E2
S31508003368200323743FE770B582B004460E460A293F
S315080033780DD06368002B08DB5D1C23441E733C2DA7
S3150800338809DC6560A3680133A36002B070BD0D212E
S31508003398FFF7E9FFEDE701AB2A4604F10C012068BF
S315080033A8FFF70BFF019B9D4202D04FF0FF35E8E778
S315080033B80025E6E730B583B0044601A9FEF7C9FC3F
S315080033C80346C8B9227C12F0200F15D012F0400F18
S315080033D80CD00123E26904F128010198407802F02B
S315080033E8D5FF88BB237C23F040032374216A019800
S315080033F8FEF7F3FC034610B1184603B030BD656AFC
S31508003408EB7A43F02003EB72A26829462068FEF798
S315080034187FFBE16805F11C00FEF72CFB0B4905F15B
S315080034281600FEF727FB002105F11200FEF71EFB22
S315080034380122019BDA700198FFF7D6FC0346227C25
S3150800344822F020022274D7E70123D5E70000614855
S3150800345810B582B00446FFF7ADFF034610B118460B
S3150800346802B010BD01A92046FEF773FC03460028E2
S31508003478F5D100222260F2E72DE9F04182B0044630
S315080034880E4601A9FEF765FC0746002840F0A2800B
S31508003498677C002F40F09E80E368B34204D2227C02
S315080034A812F0020F00D11E46636900226261002EDF
S315080034B865D0019AB2F80A804FEA482873B1721E95
S315080034C8B2FBF8F2013BB3FBF8F18A4206D3C8F11E
S315080034D8000213406361F61AA56902E0A56815B1EA
S315080034E8A56135BB4CE000212046FEF76CFF054672
S315080034F8012804D0B0F1FF3F04D0A060F0E7022706
S31508003508677467E00127677464E029462046FEF772
S3150800351815FE0546B5F1FF3F28D0012D29D9019B8F
S315080035285B699D4225D2A561636943446361A6EB3D
S31508003538080646450BD9237C13F0020FE5D0294621
S315080035482046FEF740FF05460028E3D1464663694C
S3150800355833446361C6F30803002B3FD02946019814
S31508003568FEF7B7FA40B90227677433E0012767748C
S3150800357830E0022767742DE000EB562500E00025A9
S315080035886369C3F30803E3B1E269954219D0237C5A
S3150800359813F0400F0BD0012304F128010198407855
S315080035A802F0F4FEE0B9237C23F0400323740123D8
S315080035B82A4604F128010198407802F0BDFE90B920
S315080035C8E5616369E268934204D9E360237C43F0C2
S315080035D820032374384602B0BDE8F0810025CFE7FA
S315080035E801276774F6E701276774F3E730B591B0E2
S315080035F801900D46002205A901A8FEF739FC0446E4
S3150800360810B1204611B030BD02AB0D930B4B0F938A
S31508003618019905A8FFF701FB04460028F1D10D9B7F
S3150800362893F90B30002B06DB002DEAD0294605A8AE
S31508003638FFF7BAF9E5E70624E3E700BF20150020F7
S3150800364870B59CB00190022205A901A8FEF710FCE6
S31508003658059B1193044610B120461CB070BD02ABF9
S315080036681993264B1B93019911A8FFF7D6FA044616
S315080036780028F1D1199B93F90B30002B23DB9DF811
S315080036884A3013F0010F20D10CBB059E1899304615
S31508003698FEF72BFA05469DF84A3013F0100F17D097
S315080036A806960890002106A8FEF7AEFD044678B9E6
S315080036B8002106A8FEF7E0FF034600B90723042BF6
S315080036C806D01C4604E00624DEE70724DCE70025C6
S315080036D8002CC1D111A8FFF72DF8044600B935B951
S315080036E8002CB9D10598FFF77FFB0446B4E70022FA
S315080036F8294611A8FEF7C9FE0446F1E72015002059
S315080037082DE9F04182B080460E4617460546002444
S31508003718731E9C4214DA6B46012201A93846FFF744
S3150800372893FC009B012B0BD19DF804300D2BEFD091
S315080037386A1C2B7001340A2B01D01546E8E7154692
S3150800374800232B701CB1404602B0BDE8F08100206A
S31508003758FAE710B594B0044601910023029303933F
S3150800376803E0013401A8FFF7FEFD21780029F8D106
S31508003778029A002A0CDB6B4604A90198FFF71DFD7F
S3150800378848B9009B029A9A4208D1039814B010BD0A
S315080037984FF0FF30FAE74FF0FF30F7E74FF0FF300A
S315080037A8F4E700007F2816D931B1FF2812D88038E7
S315080037B8094B33F81000704700237F2B07D8064AB1
S315080037C832F81320904202D001339BB2F5E78033D2
S315080037D8D8B270470020704764900008B0F5805F3B
S315080037E806D2224B1A881AB3904221D3F0B406E0BF
S315080037F81F4BF7E72B461A88CAB1904217D31D1DE7
S315080038085B88190ADBB29C18A04204DB0029F1D1AF
S3150800381805EB4303EFE7082909D8DFE801F0050AAD
S31508003828101316191C1F2200861A35F81600F0BC44
S315080038387047821A02F00103C01A80B2F7E71038F7
S3150800384880B2F4E7203880B2F1E7303880B2EEE784
S315080038581A3880B2EBE7083080B2E8E7503880B209
S31508003868E5E7A0F5E35080B2E1E700BF64910008F8
S315080038785893000810B4013A0A4400E0023191420C
S315080038880BD20C784B7803EB04239BB2184480B20E
S315080038988342F3D9013080B2F0E702D05DF8044BD1
S315080038A870470B781B02184480B28342F6D9013058
S315080038B880B2F3E770B4C5780D44EDB2134CE570E1
S315080038C883780E0A3344DBB2A370427862700078B4
S315080038D820709CB2A64206D90132D2B20B4C62704D
S315080038E80AB901302070C9B28D420CDA0133DBB24D
S315080038F8064A93703BB953780133DBB2537013B950
S3150800390813780133137070BC704700BF041B00207E
S3150800391810B5094C2368014603F10800FFF7CAFFEA
S315080039282368064A117819725178597291789972EA
S31508003938D278DA7210BD00BF101B0020041B0020C5
S315080039480022124B1A7006E00021114A22F81310B9
S3150800395801330E4A13700D4B1B78002BF4D0002246
S315080039680A4B1A7008E068220A4902FB031200216A
S3150800397851760133054A1370044B1B78002BF2D095
S315080039884FF48062044B1A80704700BF2017002046
S315080039987C1B0020141B0020281700200022094B36
S315080039A81A70084B1B7863B91946074A32F8132068
S315080039B81AB10133034A1370F3E7034B23F81100CE
S315080039C870477047201700207C1B0020030A43EA2B
S315080039D8002080B27047000008B514220549002067
S315080039E8FFF748FF10B94FF6FF7008BDFFF7EEFF5F
S315080039F808BD00BF9A1B002038B50D4D2B7C6C7C82
S31508003A0804EB0324A4B2143CA4B22044082205F10A
S31508003A181A0180B2FFF72EFF224605F12201FFF7A9
S31508003A2829FF10B94FF6FF7038BDFFF7CFFF38BD2D
S31508003A388C1B002008B50620FFF7DEFF08BD00002E
S31508003A4870B5994B1C68994B994A1360994A136043
S31508003A5803280DD0022800F08C80974B9B7B452BBA
S31508003A6800F038810023954A1380954A137070BD73
S31508003A78637E03F00F03032BF4D1238A002BF1D1BD
S31508003A8808228F4B1A70FDF7A7FF8D4B1B7813F08A
S31508003A98200F00F0598400238A4A1380637614227B
S31508003AA8854B83F82F202822844B1A805022824B74
S31508003AB883F82E20227A804B83F82A20627A83F8A4
S31508003AC82B20A27A83F82C20E27A83F82D20227BF1
S31508003AD883F82620627B83F82720A27B83F8282090
S31508003AE8E27B83F829200622DA75A2885A84E288B6
S31508003AF89A84754A1188598352889A832288DA8360
S31508003B0862881A84637E13F0100F00F0D6846A4B15
S31508003B18002283F8312083F83020674C4023A375A8
S31508003B28664B1B881A0A22746374002584F8355074
S31508003B3884F8345084F8325084F83350FFF77AFF03
S31508003B48C04360864523A373E573657525755F4A83
S31508003B58138801339BB213801A0AA274E374257674
S31508003B686576FFF739FFC04320830022544B1A7045
S31508003B7870BD574AD3780133DBB2D37063B99378EB
S31508003B880133DBB293703BB953780133DBB2537018
S31508003B9813B91378013313700023484A1380494A26
S31508003BA81380637E072B35D0052B33D0002B3FF4C3
S31508003BB859AF228A002A6BD0A27E511EA176002A06
S31508003BC87FF450AFE27E082A30D0591EC9B20129BF
S31508003BD82AD9042A36D803219140C9B2A1760132D6
S31508003BE8E27603F00F03013B072B3FF63BAF01A232
S31508003BF852F823F031400008513C00088D3C000873
S31508003C08C54200086D3A0008C54200086D3A000822
S31508003C18C5420008A37E0133DBB2A376782B7FF46E
S31508003C2821AF002363761DE7052AD2D100236376E0
S31508003C388022234B1A70FDF7CFFE14221E4B83F8F9
S31508003C482F2030E73021C9E700221B4B83F82F20A5
S31508003C58194B93F82F2042F0020283F82F200222EC
S31508003C6883F83620042283F83720062283F838207A
S31508003C780A2283F839202C21104A1180602283F8F9
S31508003C882E2017E704220E4B1A70FDF7A5FE80E3CF
S31508003C9803F00F03032B7FF4E5AE0822084B1A70CE
S31508003CA8FDF79AFEF1E600BF101B0020C21B002094
S31508003CB80C1B0020001B00208C1B0020FC1A00206F
S31508003CC8081B0020CE210020881B00202217002070
S31508003CD824170020B04A157C537C03EB0521AF4A0C
S31508003CE8128891423FF7BEAE8DB2AC4B1D80AA4BE7
S31508003CF81B7D13F03F0F7FF4B5AEA74B5B7D002BFA
S31508003D087FF4B0AEA64B1C880CB95B885BB1A24B96
S31508003D18DB8B9C427FF4A6AE9F4B1A8CA04B5B8824
S31508003D289A427FF49FAEFFF757FE4FF6FF73984205
S31508003D387FF498AE984BDB7D062B22D0012B7FF4B7
S31508003D4891AE954B93F82230082B7FF48BAE924BA5
S31508003D58002283F822209B8C4FF6F67293420CD9E0
S31508003D6809338D4A93848C4B5A8BDA839A8B1A8437
S31508003D785C838B4A52889A83F7E60833864A938483
S31508003D88F1E7FFF757FE4FF6FF7398427FF46AAEDE
S31508003D98844C844B9C425CD97F4B93F82F3003F0B4
S31508003DA83F03022B00F081807B4B93F82F3013F0EA
S31508003DB8040F7FF457AE784B142283F82F20282156
S31508003DC8764A1180502283F82E2093F8290093F812
S31508003DD82D2083F8292093F8281093F82C2083F8A7
S31508003DE8282083F82C1093F8272093F82B4083F87B
S31508003DF8274083F82B2093F826406B4D2C7093F8B0
S31508003E082A5083F8265083F82A400130C0B283F82E
S31508003E182D0068B94B1CDBB25F4981F82C303BB9D9
S31508003E28531CDBB281F82B3013B9013481F82A40C8
S31508003E38594B5A8C5D490A80998C59849A845A8BAD
S31508003E48DA839A8B1A84564A1188598352889A8330
S31508003E5863E6617E21B1504B9A8CA3889A4201D0B9
S31508003E68683496E74C4B5A8CE3889A42F8D14A4B01
S31508003E785A8B23889A42F3D1474B9A8B63889A427E
S31508003E88EED14B4B1C6000224A4B1A70424B93F8F2
S31508003E982F2012F0040F00F0CC800023637620222E
S31508003EA8444B1A70FDF798FDDCE53B4B9B8C99B2A1
S31508003EB83E4A138000223C4B1A7007E03E4A32F805
S31508003EC81320914207D00133374A1370364B1B78B3
S31508003ED8002BF3D068E70024334B1C703FE06824B6
S31508003EE804FB0104002C3FF4BDAD314B1C600323D1
S31508003EF8A37623760023A3750422E275E376264D76
S31508003F08AB8CA3806B8CE3806B8B2380AB8B638035
S31508003F1801206076294B1A7822735A7862739A7840
S31508003F28A273DB78E373208295F82930E37295F853
S31508003F382830A37295F82730637295F826302372CD
S31508003F48FFF7E6FC95F82E0000F0F003502B6BDD22
S31508003F580022154B1A7044E00133134A1370124BAA
S31508003F681B78002BBED1194668220E4802FB0302AD
S31508003F78527E002AB3D0072AEED13CB168220949F5
S31508003F8802FB0312917EA27E9142E5D9054A68246E
S31508003F9804FB0324E0E700BF8C1B0020FC1A002062
S31508003FA8881B0020141B0020201700202A17002031
S31508003FB8101B0020081B00207C1B0020241700204B
S31508003FC803F13601A24D695C71B3012912D00229A1
S31508003FD814D003F137029E498A5C2AB313449D4AD2
S31508003FE813709C4B1B781A4601090539B3EB810FE8
S31508003FF8E6DB19E00133974A1370F2E703F1370154
S31508004008934D695C0429E4D102F13801695C3932B7
S31508004018AB5C43EA0123904A138040F20A62934252
S3150800402828BF13466382A3821022894B83F82F2060
S315080040380EE6874B93F82E301B099B0085480370BC
S31508004048EB1A9BB2143B9BB28448038001F00F011C
S31508004058022903D102F03F0112290FD013B912F031
S31508004068030F0BD07A4BD98C2389994240F0E1810A
S31508004078774B198D6389994240F0DB8112F0100F4E
S3150800408847D0218A002944D004F10C00FFF712FC16
S315080040986F4B93F82A30724A1078834239D16C4BA1
S315080040A893F82B3051788B4233D1694B93F82C30DF
S315080040B8927893422DD1664B93F82D50684BDB784E
S315080040C89D4226D120736173A273E373E37ECBB94D
S315080040D8237EA27E9B1ADBB2A17DA3EBD103DBB2BA
S315080040E85AB21944C9B2A175002A01DA5B425AB212
S315080040F8E07DA2EB900350FA83F3DBB2E37503EB9A
S31508004108D10323760122574B1A70237EA376002300
S315080041182382617E01F00F03013B072B3FF6A2AC11
S31508004128DFE813F008002300A6006A01A101BF0111
S3150800413887015B014B4B1B7813F0010F3FF492ACD8
S31508004148032363764022474B1A7000232382434B86
S31508004158188820B14222434B1A70FFF7D9FB002270
S31508004168414B1A80FDF738FC8FE43E4B1B7813F059
S31508004178010F63D0364B93F82F3003F03F03122B09
S315080041885CD1334B93F82E0000F0F003502B2DDD4D
S315080041980022304B1A702F4B1B781A46010905392D
S315080041A8B3EB810F22DA03F13601294D695CE9B1CF
S315080041B8012903D10133274A1370ECE7022933D1C1
S315080041C803F13701224D695C04292DD102F1380122
S315080041D8695C3932AB5C43EA01231F4A138040F213
S315080041E80A62934228BF13466382A382032363762F
S315080041F8174B93F82620227293F82720627293F8B1
S315080042082820A27293F82930E3720120FFF780FB71
S315080042184222144B1A7000232382104A1380124A2A
S315080042281380FDF7D9FB30E403F1370208498A5CA5
S31508004238002ADBD01344074A1370ACE72022094B3F
S315080042481A70FDF7C9FB094B1B6800225A76ABE5BD
S315080042588C1B0020201700202A170020FC1A002093
S31508004268041B0020081B0020CE210020101B00205C
S31508004278964B93F82F3013F0010F25D011F0100F35
S3150800428822D1238A002B7FF4EDAB914D2888013083
S3150800429880B2FFF73DFB8F4A137843F0100313707B
S315080042A82A881AB143F002038A4A1370FDF794FB69
S315080042B801232382082363760023E3761122834B9E
S315080042C883F82F20FFF7EFBB13F0200F0FD07F4896
S315080042D890F834301A0290F8353042EA03067E4DD3
S315080042E82868304428607A480288931B0380784BEC
S315080042F8188848B111F0100F06D1764A137843F09A
S3150800430802031370FFF704FB704B93F8302093F8F9
S31508004318313003EB02239BB2704A1380A28A934278
S3150800432800D80BB96D4B1A806C4B1B886382694B96
S315080043381B7813F0030F3FF495AB0022684B1A80DD
S31508004348FDF74AFBFFF7A1BB13F0100F0DD00023AA
S31508004358634A13800122228204226276E3761122B6
S315080043685A4B83F82F20FFF79EBB5D4A128872B115
S3150800437813F0010F01D000232382238ADBB9638A4D
S315080043889A4201D9564A1380554B1B882382002323
S31508004398E376544B1A68504B1A60514B1B886BB11D
S315080043A8238A5BB128334A4A13801822474B83F875
S315080043B82F20FFF77BBB4A4A1380E8E7454B1B7853
S315080043C813F0020F3FF44EAB2822414B1A801022F5
S315080043D83E4B83F82F20FFF769BB3E4B1B7813F03B
S315080043E8010F3FF43FAB002363761022394B1A704E
S315080043F8FDF7F2FAFFF736BB354B188808B1FFF711
S3150800440887FA324B93F82F3013F0010F1AD0314B35
S315080044181B7813F0010F12D0072363760023A376BF
S3150800442823820120FFF774FA10222A4B1A70FDF727
S31508004438D3FA1022254B83F82F20FFF734BB06231F
S315080044486376EEE7234B1B7813F0010F05D0052397
S31508004458637600232382FFF705BB1D4B1B88002BB9
S31508004468E7D1FFF7FFBA1A4B188808B1FFF750FAD1
S31508004478164B93F82F3013F0010F0CD007236376E9
S315080044880023A3760120FFF743FA1022114B1A706E
S31508004498FDF7A2FACDE70E4B1B88002BC9D1FFF70B
S315080044A8E1BA0C4B1B7813F0010F3FF4DBAA07237C
S315080044B863760023A376FFF7D5BA044B062283F85A
S315080044C830200A2283F83120FFF727BB8C1B0020EF
S315080044D8FC1A0020081B00200C1B00202A170020A5
S315080044E8CE210020001B002000290CDD08B58AB261
S315080044F8054B1A80054B1B68834203D001461846AC
S3150800450804F0ACFB08BD7047CE210020001B002034
S31508004518F0B40022394B1A7002E00133374A137097
S31508004528364B1B78072B18D8354D5A001A44940071
S315080045382E192A5B002AF0D07488002CEDD005883D
S31508004548AA42EAD142889442E7D10C6874608988FD
S3150800455831812C4B1B78B37222E00022274B1A7044
S3150800456802E00133254A1370244B1B78072B0AD817
S31508004578234D5A001A4494002E192A5B002AF0D1B2
S315080045887288002AEDD1082B0CD00268334643F806
S31508004598042B0A6872608A889A801A4B1B78B37249
S315080045A8F0BC70470023184A1370184A1370134A48
S315080045B8137002E00133114A1370104B1B78072B4E
S315080045C811D8104A147803EB430295000C4A2A447A
S315080045D8927AA61A0C4D2D78AE42EBDD0A4A167069
S315080045E80A4A1370E6E7094B1B78044A137003EB6B
S315080045F843039A00024E1644C7E700BF96170020E1
S3150800460834170020941700209C17002095170020BF
S3150800461810B4164B1C780134E4B21C700022144BF3
S315080046281A7002E00133124A1370114B1B78072BD4
S3150800463818D810485A001A4491004218415A528804
S315080046480A43EFD003EB4302910002460A44927AE2
S31508004658A21A772AE6DD03EB43018A0000200549FA
S315080046688850DFE75DF8044B704700BF94170020B1
S315080046789617002034170020334B1B88292B0CD992
S3150800468810B50022304B1A80304B9B8AB3F5807FD1
S3150800469807D0B3F5007F44D010BD00222A4B1A80F4
S315080046A870472A4BDA8C2A4B1B889A4200D010BDD1
S315080046B8264B1A8D264B5B889A42F8D1254C2146FB
S315080046C8A01DFFF725FF002204F8022C022204F891
S315080046D8012C2168C4F80A10A188E1811E490868D6
S315080046E820608988A18044F8100C24F80C1CD4F89A
S315080046F80A1044F8161CE28924F8122CE288228249
S3150800470822896282124A1188E18052882281082207
S3150800471804F80A2C062204F8092C2A220A4B1A80BD
S3150800472810BD0A4BDA8C0A4B1B889A42BFD1074B35
S315080047381A8D074B5B889A42B9D106480146063056
S31508004748FFF7E6FEB3E700BFFC1A00208C1B002023
S31508004758881B0020A21B00202C17002030B4484BC9
S31508004768DA8B4FF6FF739A4219D0464B1B8846498F
S3150800477809885340194208D1414B198C414B5B882B
S31508004788414840884B40184216D0404B404A118849
S31508004798198052885A8000223E4B1A7013E0384B0B
S315080047A8198C4FF6FF739942DFD1354B3A4A106890
S315080047B8186092889A8021E0344B1A805980EAE773
S315080047C80133344A1370334B1B78072B0ED83348FA
S315080047D85A001A44910045182C4A1488425A944299
S315080047E8EED12A4A50886A889042E9D1082B16D011
S315080047F8234B55F8042F1A60AA889A80204B284A12
S315080048081168C3F8061092885A8108221A7300227A
S315080048185A73244A13880E33138030BC7047184BD2
S315080048284FF0FF321A609A8000221A629A841C494D
S315080048380868C3F8060089885981C3F81600598399
S3150800484812490888D884498819850E49088898839A
S315080048584988D9831A75012159759A73D973082114
S3150800486819745A7406229A740422DA741973062279
S315080048785A7336330C4A13602A220A4B1A80CCE735
S315080048888C1B0020881B0020841B002098170020FA
S31508004898801B00209617002014940008341700205F
S315080048A82C170020FC1A00200C1B00200022014BA4
S315080048B85A707047A0170020034BFE22DA70187149
S315080048C80222A3F844207047A017002010B5054C0B
S315080048D800232370FFF7EAFFFF23E3700123A4F8F8
S315080048E8443010BDA0170020064BFF22DA700022BC
S315080048F81A71597859719A71DA711A720622A3F8D7
S3150800490844207047A017002008B50020FFF7D4FFF9
S3150800491808BD0000074BFF22DA70074A9A6400228E
S315080049281A715A719A710722C3F807200822A3F840
S3150800493844207047A01700201C940008044BFF2247
S31508004948DA7042689A640122A3F84420704700BFC7
S31508004958A017002008B53120FFF7AEFF08BD0000F4
S3150800496838B5084CFF23E370002525716571FCF7F7
S315080049788DFBA071E571257265720723A4F844308A
S3150800498838BD00BFA017002038B5FCF72DFCE8B1E4
S31508004998FFF78CFF0F4C01252570FF23E3701023C2
S315080049A8237100236371FCF771FBA071FCF77CFB8C
S315080049B8E071FCF779FBC0F3072020726572A572CF
S315080049C80823A4F84430FBF78FFF38BD1020FFF7FB
S315080049D873FF38BDA017002038B505464478FCF79C
S315080049E855FB0138844210DC0A4C6A78A16C201DF4
S315080049F8FBF78EFDFF23E3706A78A36C1344A36460
S31508004A086B780133A4F8443038BD2220FFF754FFE9
S31508004A1838BD00BFA017002038B504464578FCF70E
S31508004A2835FB0138854211DC61680A4DA96462784C
S31508004A38281DFBF76DFDFF23EB706278AB6C1344FA
S31508004A48AB6463780133A5F8443038BD2220FFF7F4
S31508004A5833FF38BDA0170020F8B5054617460024C9
S31508004A6806E015F8013B1C44E4B2FCF730FB314676
S31508004A784E1E0029F5D13C600120F8BD10B5084C3A
S31508004A88FF23E370E21D4168A06CFFF7E5FF20717C
S31508004A9800236371A3710823A4F8443010BD00BF2E
S31508004AA8A017002038B505460D4B9C6CFCF7EEFAA6
S31508004AB86A1C411E2046FBF71BFF60B1084CFF2302
S31508004AC8E370FCF7E3FA0138A36C0344A3640123F3
S31508004AD8A4F8443038BD3120FFF7EEFE38BD00BFD4
S31508004AE8A017002038B504464578FCF7CFFA0238EF
S31508004AF885420EDC114BFF22DA700122A3F8442006
S31508004B08617851B9FBF704FF90B93120FFF7D4FE55
S31508004B1838BD2220FFF7D0FE38BDA21C074B986C7B
S31508004B28FBF7E6FE28B16178044A936C0B44936454
S31508004B3838BD3120FFF7C0FE38BD00BFA0170020DA
S31508004B4808B54168074B986CFBF7D6FE30B1054B9C
S31508004B58FF22DA700122A3F8442008BD3120FFF7A6
S31508004B68ABFE08BDA017002008B5FBF7B3FC034B3E
S31508004B78FF22DA700122A3F8442008BDA0170020F6
S31508004B8808B589B2FCF758FA08BD0000054B00229B
S31508004B981A709A6483F84320A3F844209A705A70C6
S31508004BA8704700BFA0170020034B1B780BB10120E4
S31508004BB870470020704700BFA01700200022024B4C
S31508004BC883F84320704700BFA017002008B503786C
S31508004BD8FF2B04D0354A1278012A14D008BDFFF7EE
S31508004BE8D3FE324B93F84330012B5AD02F4BB3F9E7
S31508004BF844100029F2DD1846012380F843300330B3
S31508004C08FFF7BEFFEAE7C93B352B46D8DFE803F0CE
S31508004C183345454245453F363C394545454545456D
S31508004C28454545454545454545454545454545451E
S31508004C3845454545454545454545241E1B214545A4
S31508004C484527452A2D30FFF7C7FECAE7FFF7E4FED2
S31508004C58C7E7FFF773FEC4E7FFF710FFC1E7FFF7DB
S31508004C6859FEBEE7FFF750FEBBE7FFF73DFEB8E77C
S31508004C78FFF72CFEB5E7FFF715FFB2E7FFF732FF98
S31508004C88AFE7FFF76DFEACE7FFF75AFFA9E7FFF7AF
S31508004C986BFFA6E7FFF75EFEA3E72020FFF70CFEEB
S31508004CA89FE71020FFF708FEA0E700BFA01700201F
S31508004CB8704770477047000008B50121044801F09D
S31508004CC83EFD012801D0012008BD002008BD00BF0F
S31508004CD80000024000B5C7B04FF48C720021684640
S31508004CE803F0C7FF69460948FEF780FC40B9009BF0
S31508004CF853B19DF8083013F0100F02D1012000E0D7
S31508004D08002047B05DF804FB0020FAE73494000851
S31508004D18004870473494000808B50748002380F807
S31508004D2828320A220549FEF7D1F818B90122024B9A
S31508004D3883F8282208BD00BFEC1700202494000831
S31508004D4810B50D4B93F82832012B10D0FBF714FE3B
S31508004D5800F164044021094801F0DCFE18B9FBF7A4
S31508004D680BFE8442F6D20648FEF76AFC10BD0248D6
S31508004D78FEF76EFBEAE700BFEC17002000140140B7
S31508004D883494000808B5054B93F82832012B00D04F
S31508004D9808BD0248FEF75CFBFAE700BFEC170020DF
S31508004DA810B504460F4B93F82832012B15D10D4937
S31508004DB8FEF7CFFC002810DA0A48002380F82832C4
S31508004DC8FEF746FB09E0084801F09CFE80210648E4
S31508004DD801F0A0FE0028F9D0013421780029F2D183
S31508004DE810BD00BFEC1700200014014008B50121CA
S31508004DF84FF0007001F056FD00214FF0007001F0E9
S31508004E0851FD08BD0023036043608360C3600361E6
S31508004E1843618361C361036243628362C362036356
S31508004E2843638363C3634022026420224264836423
S31508004E38C364036543658365C36503668022426662
S31508004E488366C366036743678367C3674FF08062F1
S31508004E58C0F880204FF00072C0F884204FF08071A7
S31508004E68C0F888104FF40011C0F88C10C0F89030BC
S31508004E78C0F89430C0F89830C0F89C30C0F8A03014
S31508004E88C0F8A420C0F8A8304FF40032C0F8AC2007
S31508004E984FF48072C0F8B020C0F8B430C0F8B83003
S31508004EA87047000082B000230193124A136903F081
S31508004EB81C03C00280B20343890101F4F8610B435D
S31508004EC843F001031361019B01330193094B1B69E5
S31508004ED813F0010F03D0019A074B9A42F3D9019AA6
S31508004EE8064B9A4204D0034B586980B202B0704701
S31508004EF80020FBE700800240FEFF0400FFFF0400D5
S31508004F0810B483B000230193124C236903F01C03E1
S31508004F18C00280B20343890101F4F8610B4343F0E8
S31508004F28030362612361019B01330193094B1B69E2
S31508004F3813F0010F03D0019A074B9A42F3D9019A45
S31508004F48064B9A4204D0012003B05DF8044B70471B
S31508004F580020F9E700800240FEFF0400FFFF040076
S31508004F6870B586B004460D46002305930093924B08
S31508004F781E6926F01C0601A801F000FC029A8F4B50
S31508004F8813448F498B4211D846F008068A4B1E618E
S31508004F984FF4004200212846FFF7B2FF03460028CF
S31508004FA800F003814FF08063059312E0854B1344A4
S31508004FB885498B4202D846F00C06E7E7834B13442B
S31508004FC8834A9342E2D946F00406DFE7059B013B8C
S31508004FD80593059B002BF9D12368002B49D0009B24
S31508004FE80133009301212846FFF75CFF10F0040FF0
S31508004FF803D1009A774B9A42F1D9009A764B9A428E
S3150800500800F0D680002100914FF480522846FFF719
S3150800501877FF0346002800F0C880009B01330093F9
S3150800502801212846FFF73EFF10F0200F03D1009A0A
S31508005038684B9A42F1D9009A674B9A4200F0BA80AF
S315080050480023009310212846FFF72CFF10F0040FC1
S3150800505808D04FF40063236210F0020F05D000232E
S3150800506863611FE000232362F6E74FF48043636118
S3150800507818E0226AC2F3CF026369C3F34F031A43DF
S3150800508800212846FFF73CFF0346002800F08D80DC
S315080050986FF07F43059302E0059B013B0593059B4B
S315080050A8002BF9D1444A13684C4919406368A0682B
S315080050B80343E06803432069034360690343A0691F
S315080050C80343E0690343206A0343606A0343A06A0B
S315080050D80343E06A0343206B0343606B03430B43B4
S315080050E81360A36BE16B0B43216C0B43616C0B4399
S315080050F8A16C0B43E16C0B43216D0B43616D0B43AC
S315080051085360A36D9360E36DD360916921F0BE0186
S315080051180904090C206E636E43EA0043A06E034334
S31508005128E06E0343206F0343606F03430B439361A9
S31508005138A36FE16F0B43D36141F21800135828494E
S315080051481940D4F88030D4F884502B43D4F88850C2
S315080051582B43D4F88C502B43D4F890502B43D4F8CF
S3150800516894502B43D4F898502B43D4F89C502B438F
S31508005178D4F8A0502B430B431350D4F8A430D4F8D2
S31508005188A8100B43D4F8AC100B43D4F8B0100B4353
S31508005198D4F8B41043EA8103D4F8B8100B4343F49F
S315080051A8000302F5805213600123184606B070BD45
S315080051B80023FAE70023F8E70080024000D3CEFE72
S315080051C8BFE1E40040F1E9FD3F787D0100796CFC18
S315080051D8005A6202FEFF0400FFFF04000F8120FF49
S315080051E8233FDEF828B9064A136823F00803136034
S315080051F87047034A136843F008031360704700BFF3
S315080052080080024028B9064A136823F0040313608D
S315080052187047034A136843F004031360704700BFD6
S3150800522800800240024A136843F00103136070477E
S3150800523800900240044B1B6813F0010F01D10020AF
S3150800524870470120704700BF00900240034941F2A9
S3150800525818028B5843F480138B507047008002401D
S3150800526838B9084941F218028B5823F400538B5071
S315080052787047044941F218028B5843F400538B507F
S31508005288704700BF0080024038B9084941F2180241
S315080052988B5823F002038B507047044941F21802D1
S315080052A88B5843F002038B50704700BF00800240BA
S315080052B808B50120FFF796FFFFF7C8FF0120FFF79B
S315080052C8A1FF0120FFF7CCFF0120FFF7DDFF08BD8E
S315080052D82DE9F04182B001210C2001F0ABFA2C4CE3
S315080052E80C220821204601F031FA0C220921204611
S315080052F801F02CFA0C220A21204601F027FA0C2282
S315080053080B21204601F022FA0C221146204601F00C
S315080053181DFA204F0C220221384601F017FA4FF4DD
S315080053287063009301258DF805504FF002088DF833
S31508005338048000268DF806608DF8075069462046D1
S3150800534801F0B8F9042300936946384601F0B2F922
S315080053584FF4805300938DF807606946204601F09C
S31508005368A9F94FF4006700978DF804808DF807604F
S315080053786946204601F09EF92946384601F084FA1E
S3150800538829464FF4800001F055FA02B0BDE8F081CD
S3150800539800080240000C024010B54FF4803400E0C3
S315080053A8013C24B1802001F021FB0028F8D00CB973
S315080053B8032010BD40F2FF5001F022FB002010BD6B
S315080053C808B5104B5A6B4FF4803302E0013B0D4A7F
S315080053D8526B12F0450F01D1002BF7D113B112F019
S315080053E8040F04D0042001F00BFB032008BD12F0BB
S315080053F8400F01D1002008BD402001F001FB002024
S3150800540808BD00BF002C014008B50B4B5B6B01E0DB
S31508005418094B5B6B13F0450FFAD013F0040F04D051
S31508005428042001F0EDFA032008BD40F2FF5001F010
S31508005438E7FA002008BD00BF002C014008B50F4B4D
S315080054485B6B01E00D4B5B6B13F0450FFAD013F05D
S31508005458040F08D113F0010F0AD140F2FF5001F0EA
S31508005468CFFA002008BD042001F0CAFA032008BDB7
S31508005478012001F0C5FA012008BD00BF002C014033
S3150800548810B50446454B5B6B01E0444B5B6B13F068
S31508005498450FFAD013F0040F08D113F0010F0AD1FB
S315080054A801F06EFAA0420BD0102010BD042001F0BE
S315080054B8A7FA032010BD012001F0A2FA012010BDA9
S315080054C840F2FF5001F09CFA002001F05FFA344BD5
S315080054D80340002B3FD000283FDB10F0804F01D057
S315080054E8092010BD10F0005F01D00A2010BD10F089
S315080054F8805F01D00B2010BD10F0006F2FD110F07F
S31508005508806F2ED110F0807F2DD110F4000F2CD18A
S3150800551810F4800F2BD110F4001F2AD110F4801F25
S3150800552829D110F4002F28D110F4802F27D110F490
S31508005538003F26D110F4803F25D110F4004F24D11E
S3150800554810F4804F23D110F4005F22D110F0080F11
S3150800555821D01A2010BD002010BD1C2010BD0C201B
S3150800556810BD0D2010BD0E2010BD0F2010BD102037
S3150800557810BD112010BD122010BD132010BD142017
S3150800558810BD152010BD162010BD172010BD1820F7
S3150800559810BD192010BD002010BD00BF002C014009
S315080055A808E0FFFD38B504460D461E4B5B6B01E067
S315080055B81C4B5B6B13F0450FFAD013F0040F08D198
S315080055C813F0010F0AD101F0DBF9A0420BD0102025
S315080055D838BD042001F014FA032038BD012001F073
S315080055E80FFA012038BD40F2FF5001F009FA0020F1
S315080055F801F0CCF910F4604F04D010F4005F05D020
S31508005608132038BD000C2880002038BD10F4804FC0
S3150800561801D0102038BD10F4004F01D00F2038BD36
S31508005628002038BD002C0140F0B583B00D46002394
S3150800563800930193564808220260102444604022C9
S315080056488260C3604FF48063036101F081F92046E4
S31508005658FFF716FF064610B1304603B0F0BD4D4BAE
S315080056681B68A3404A480360372444604023836084
S315080056780023C3604FF48063036101F069F920468B
S31508005688FFF7FEFE06460028E6D143484FF0FF33EB
S31508005698036008234360302383600223C360002421
S315080056A804610123436101F07DF939480460332612
S315080056B8466040238360C4604FF48063036101F049
S315080056C847F93046FFF7DCFE06460028C4D12746C8
S315080056D804E0013442F210739C4256D82F4B5A6B99
S315080056E840F22A631A420BD14FF4001001F07EF9F2
S315080056F80028EED001F06EF94DF827000137E8E7E3
S31508005708082001F073F920B1082001F079F9042678
S31508005718A2E7022001F06AF920B1022001F070F927
S31508005728022699E7202001F061F920B1202001F02E
S3150800573867F9062690E74FF4007001F057F928B183
S315080057484FF4007001F05CF9072685E740F2FF5030
S3150800575801F056F9009A130203F47F0343EA026339
S31508005768110A01F47F410B4343EA12636B60019AFD
S31508005778130203F47F0343EA0263110A01F47F4123
S315080057880B4343EA12632B6066E7042664E700BF07
S31508005798981A00203C1A0020AC1A0020002C014058
S315080057A810B582B0044600200090019001F0EEF88A
S315080057B810F0007F03D00E23184602B010BD6946C4
S315080057C8324B1888FFF730FF03460028F4D1012C1E
S315080057D805D0019B13F4803F30D12523ECE7019BC4
S315080057E813F4802F01D12523E6E7284B1B681B04F1
S315080057F82748036037244460402383600023C36036
S315080058084FF48063036101F0A3F82046FFF738FEDA
S3150800581803460028D0D11E480223036006244460A4
S31508005828402383600023C3604FF48063036101F05B
S315080058388FF82046FFF724FE0346BDE7134B1B687F
S315080058481B041348036037244460402383600023FD
S31508005858C3604FF48063036101F07AF82046FFF7C6
S315080058680FFE03460028A7D109480023036006242B
S31508005878446040228260C3604FF48063036101F08C
S3150800588867F82046FFF7FCFD034695E73C1A002013
S31508005898981A002000B583B001238DF807304FF415
S315080058A80061064800F04BFF10B900238DF8073051
S315080058B89DF8070003B05DF804FB00BF0008024026
S315080058C870B582B000248DF80740634876230375BF
S315080058D8046044608460C460046101F00BF8032026
S315080058E801F028F8012001F01FF85C4804604460BC
S315080058F88460C4604FF48063036101F029F8FFF7F8
S315080059084BFD8DF807009DF8073023B19DF8070071
S31508005918C0B202B070BD51484FF4D573036008236E
S315080059284360402383600023C3604FF480630361A8
S3150800593801F00EF8FFF744FD8DF807009DF80730CB
S31508005948EBB90122464B1A604FF0804643480023BC
S3150800595803603724446040228260C3604FF4806342
S31508005968036100F0F5FF2046FFF78AFD8DF807006A
S315080059789DF80730F3B19DF80700C0B2C9E7374864
S31508005988002606603724446040238360C6604FF4C7
S315080059988063036100F0DCFF2046FFF771FD8DF890
S315080059A80700D3E79DF80700C0B2B2E79DF80700DD
S315080059B8C0B2AEE7002004460246002839D14FF6A1
S315080059C8FE739C4235D82548002303603725456071
S315080059D840228260C3604FF48063036100F0B8FF19
S315080059E82846FFF74DFD8DF807009DF80730002B70
S315080059F8D8D146F0004343F4801318480360292396
S31508005A084360402383600023C3604FF480630361C7
S31508005A1800F09EFFFFF7F8FC8DF807009DF80730A1
S31508005A28002BC3D1002000F0B1FF0246C00F013495
S31508005A38C3E74FF6FE739C4206D812F0804F9AD0F9
S31508005A480222074B1A6096E71B238DF807309DF844
S31508005A580700C0B25DE700BFC41A0020981A0020E4
S31508005A68381A002030B583B00123ADF8063000F0A7
S31508005A7867FF18B92524204603B030BD384B1B6884
S31508005A88042B21D037480023036002224260C02233
S31508005A988260C3604FF48063036100F059FFFFF723
S31508005AA8CDFC04460028E6D100F070FF2E4C206095
S31508005AB8042000F06BFF6060082000F067FFA06014
S31508005AC80C2000F063FFE060254B1B68012B2FD9DB
S31508005AD8062B2DD0022B2BD0214B1B68042B3DD02F
S31508005AE8BDF80630214A13601B041E4803600923C3
S31508005AF84360C02383600023C3604FF48063036157
S31508005B0800F026FFFFF79AFC04460028B3D100F0F8
S31508005B183DFF174D2860042000F038FF686008200C
S31508005B2800F034FFA8600C2000F030FFE860A2E718
S31508005B380C48002303600324446040228260C36043
S31508005B484FF48063036100F003FF0DF10601204658
S31508005B58FFF728FD04460028BED08CE700248AE70C
S31508005B68381A0020981A0020181A00203C1A002013
S31508005B78281A0020F0B40346A24A146880F856404A
S31508005B88A14A1288A0F85420A04D2A68100EC1B25E
S31508005B988E091E70C0F38300587001F003019970CE
S31508005BA8C2F30741D970C2F307211971D2B25A71E3
S31508005BB869680A0E1201DA80C1F30740DA8892B2D8
S31508005BC842EA1012DA8000F00F001872080AC2B208
S31508005BD8D5095D72C0F380159D72C0F34015DD7254
S31508005BE8C0F300151D7300255D73012C40F2A980CA
S31508005BF8022C00F0E680C2F380115976520002F0B2
S31508005C087E029A768148027A997E41EAD211997675
S31508005C1802F07F02DA76C1680A0ED0091877C2F34D
S31508005C2841105877C2F382009877920002F00C0266
S31508005C38DA77080CC2B2DC7F44EA9214DC77C0F340
S31508005C48401083F82000002083F8210002F00102A2
S31508005C5883F822200A0AD4B2E50983F82350C2F346
S31508005C68801583F82450C2F3401583F82550C2F3EB
S31508005C78001583F82650C2F3810283F8272004F01A
S31508005C88030483F82840C1F3460183F82910012440
S31508005C9883F82A405E4D2A68110E83F82C10C2F341
S31508005CA807410902D985C2F30726D98D89B2314336
S31508005CB8D98512061A636A68160E196B41EA0641EF
S31508005CC81963110C1E6B090289B2314319631E6BDD
S31508005CD8C2F3072131431963D2B283F83420AA687C
S31508005CE8110E83F83510110C09069963110A9E6B73
S31508005CF8090401F47F0131439963996B120292B240
S31508005D080A439A63EA68996B41EA12619963110C26
S31508005D1893F83C50C1F30316354383F83C500902FF
S31508005D2801F47061D987C2F30725D98F89B2294347
S31508005D38D987C2F3460283F8402083F84140F0BC6D
S31508005D487047800200F4406018611A69890001F4F6
S31508005D587F71114319612D4A9268100EC1B21C69E8
S31508005D6844EA91141C61C0F3C200187501F00701D2
S31508005D785975110CC1F342109875C1F38200D8758C
S31508005D88490001F006011976C2F30722197E41EA8D
S31508005D98D21119761D690135187E0230012404FAD4
S31508005DA800F0C717A5FB000105FB07111D7AEDB220
S31508005DB8AC401C65A0FB046704FB0177C3E91267BE
S31508005DC819E7090401F47C111961104A9268100E42
S31508005DD8196941EA002119611869C2F307410143A3
S31508005DE81961C2F3072218690021013041F100013F
S31508005DF8C90441EA5031C0049864D9644FF4007163
S31508005E081965F8E6381A00203C1A0020281A0020D6
S31508005E18181A002010B51A4B1B68032B29D0022B19
S31508005E282AD8B0F5805F29D0B0F5006F0FD00020CA
S31508005E38FFF7B6FC0446E8B9124800230375036061
S31508005E4843608360C360036100F054FD12E00120DB
S31508005E58FFF7A6FC044668B90A48002303750360D9
S31508005E68436083604FF40062C260036100F042FD3C
S31508005E7800E02724204610BD0024FBE72724F9E77D
S31508005E88381A0020C41A002010B5094B18600724D0
S31508005E985C6040229A600022DA604FF480621A61D8
S31508005EA8184600F055FD2046FFF7EAFA10BD00BF70
S31508005EB8981A002000B583B000238DF80730FFF73D
S31508005EC807FA00F00BFDFFF7FBFC8DF807009DF8B5
S31508005ED807302BB19DF80700C0B203B05DF804FB84
S31508005EE8FFF7C0FD8DF807009DF807301BB19DF830
S31508005EF80700C0B2F1E7154800230375036043603D
S31508005F088360C360036100F0F5FC1148FFF732FEB1
S31508005F188DF807009DF8073033B19DF807306BB147
S31508005F289DF80700C0B2D8E7094BB3F85400000437
S31508005F380021FFF7A9FF8DF80700EEE74FF4006088
S31508005F48FFF768FF8DF80700EAE700BFC41A0020C4
S31508005F58401A00202DE9F04105461646BDF81810E6
S31508005F680022534802705348026053480260534857
S31508005F78C262534A1268022A10D0884651480160FC
S31508005F8810234360402383600023C3604FF4806373
S31508005F98036100F0DDFC4FF4803406E0720A42EA39
S31508005FA8C3564FF40071E8E7013C24B1802000F09D
S31508005FB81DFD0028F8D01020FFF762FA074610B131
S31508005FC83846BDE8F08140484FF0FF330360C0F813
S31508005FD80480902383600223C36000270761012396
S31508005FE8436100F0DFFC374806601124446040230B
S31508005FF88360C7604FF48063036100F0A9FC2046FC
S31508006008FFF73EFA07460028DAD12C4B5A6B40F2BE
S315080060182A631A4210D14FF4004000F0E7FC002822
S31508006028F3D0002404E000F0D5FC45F82400013438
S31508006038072CF8D92035E8E7082000F0D7FC20B166
S31508006048082000F0DDFC0427BAE7022000F0CEFCA1
S3150800605820B1022000F0D4FC0227B1E7202000F086
S31508006068C5FC20B1202000F0CBFC0627A8E74FF492
S31508006078007000F0BBFC68B94FF0FF344FF400100D
S3150800608800F0B4FC60B15CB100F0A4FC45F8040B60
S31508006098013CF3E74FF4007000F0B2FC07278FE7DE
S315080060A840F2FF5000F0ACFC0022084B1A6087E764
S315080060B8E41A0020E01A0020DC1A0020002C01400F
S315080060C8381A0020981A0020AC1A0020040000206C
S315080060D82DE9F04106461546BDF818100022534822
S315080060E8027053480260534802605348C262534AD2
S315080060F81268022A15D0884651480160102444605F
S31508006108402383600023C3604FF48063036100F073
S315080061181FFC2046FFF7B4F9074640B13846BDE8E4
S31508006128F0816A0A42EAC3554FF40071E3E7444826
S31508006138056018244460402383600023C3604FF435
S315080061488063036100F004FC2046FFF799F90746C7
S315080061580028E3D13B484FF0FF330360C0F80480BA
S31508006168902383600024C46004610123436100F01E
S3150800617819FC314B5A6B40F21A631A422CD14FF468
S31508006188804000F033FC0028F3D0C4F50078B8F155
S315080061981F0F1FD8634213F0030F03D14FEA98085D
S315080061A800250AE04FEA980808F10108F8E756F8C2
S315080061B8040B00F015FC013504344545F7D3D8E738
S315080061C856F8250000F00CFC0135072DF8D92036BD
S315080061D82034CEE70025F8E7082000F007FC20B1B0
S315080061E8082000F00DFC042798E7022000F0FEFBC3
S315080061F820B1022000F004FC02278FE7102000F0E7
S31508006208F5FB20B1102000F0FBFB052786E74FF4C5
S31508006218007000F0EBFB18B900220B4B1A607DE7FB
S315080062284FF4007000F0ECFB072777E7E41A002024
S31508006238E01A0020DC1A0020002C0140381A002039
S31508006248981A0020AC1A00200400002038B5C8B1F6
S3150800625805460E4B1B681B040D4803600D24446055
S31508006268402383600023C3604FF48063036100F012
S315080062786FFB2046FFF704F9044620B900F086FBB1
S31508006288286000E02624204638BD00BF3C1A0020B6
S31508006298981A002000B583B000230193FFF7FAFA8D
S315080062A8012803D0FF2003B05DF804FB01A8FFF717
S315080062B8CDFF08B1FF20F6E70198C0F34320F2E7BF
S315080062C808B5FFF7E7FF042805D0FF2801D0012005
S315080062D808BD022008BD002008BD704770470000A9
S315080062E800B597B0FFF7E6FD30B10122074B1A70E3
S315080062F8032017B05DF804FB044A137803F0FE037D
S3150800630813706846FFF736FC0020F2E708000020FD
S3150800631808B50122074B1A7010B1064B187808BD44
S31508006328FFF7CEFF0028F8D1024A137803F0FE03D8
S315080063381370F2E70800002070B5ADF5027D0E4629
S315080063481546E8B95C1ECBB162194FF40073009381
S315080063585202002302A8FFF7FDFDA8B9FFF7B0FF10
S315080063680128FBD04FF4007202A906EB442002F07C
S3150800637875FC2346002CE5D1002002E0012000E048
S3150800638801200DF5027D70BD0120FAE7F0B5ADF5DF
S31508006398037D0F46164648B101200DF5037DF0BD6D
S315080063A8FFF78EFF0128FBD02346C4B15C1EA3B1B4
S315080063B84FF400752A4607EB442102A802F04EFC62
S315080063C8A21900955202002302A8FFF781FE0028A9
S315080063D8E6D00528E4D00120DFE70120DDE7002024
S315080063E8DBE70000164B1B7813F0010F01D00320DA
S315080063F87047032920D8DFE801F00204161B00209D
S31508006408704708B10020704710B596B0144668461C
S31508006418FFF7B0FB129B5B0A139A43EAC253236041
S31508006428002016B010BD4FF4007313800020704783
S3150800643820B920231360704704207047002070474E
S315080064480800002082B00023019300932A4A1368A3
S3150800645843F480331360284B1B6803F40033009316
S31508006468019B01330193009B1BB9019BB3F5A06FF0
S31508006478F1D1214B1B6813F4003F06D00123009382
S31508006488009B012B04D002B0704700230093F7E75E
S31508006498194B1A6C42F080521A6418490A6842F471
S315080064A840420A609A689A609A6842F400429A607A
S315080064B89A6842F4A0529A60114A5A601A6842F0D9
S315080064C880721A600C4B1B6813F0007FFAD040F2F2
S315080064D805620C4B1A60A3F580639A6822F00302DA
S315080064E89A609A6842F002029A60034B9B6803F026
S315080064F80C03082BF9D1C6E70038024000700040A3
S315080065080C544007003C024010B5104CD4F88830AB
S3150800651843F47003C4F888300D4B1A6842F0010238
S315080065281A60002199601A6822F0847222F480326F
S315080065381A60084A5A601A6822F480221A60D960D2
S31508006548FFF780FF4FF00063A36010BD00ED00E081
S315080065580038024010300024054B1B69002B00DB6D
S315080065687047034B034A5A6002F188325A60F7E7C4
S31508006578003C024023016745024A136943F0004379
S3150800658813617047003C0240014BD860704700BF52
S31508006598003C02400E4BDB6813F4803F14D10C4BC9
S315080065A8DB6813F0100F01D005207047084BDB682D
S315080065B813F0EF0F01D006207047054BDB6813F080
S315080065C8020F03D00720704701207047082070473C
S315080065D8003C024000B583B008238DF80730FFF762
S315080065E8D9FF8DF8070003E0FFF7D4FF8DF80700F9
S315080065F89DF80730DBB2012BF6D09DF8070003B0EB
S315080066085DF804FB70B5064649B101290DD0022983
S3150800661802D04FF4407503E04FF4007500E00025FA
S31508006628FFF7D8FF082803D070BD4FF48075F7E741
S315080066380F4C236923F44073236123691D4325619D
S31508006648236923F0F803236123691E4346F00206EB
S315080066582661236943F480332361FFF7BBFF236967
S3150800666823F002032361236923F0F8032361DBE798
S31508006678003C024070B505460E46FFF7ABFF0828F2
S3150800668800D070BD0A4C236923F44073236123693B
S3150800669843F400732361236943F0010323612E60E1
S315080066A8FFF798FF236923F001032361E9E700BF91
S315080066B8003C024000230F2B40D8F0B425E084683C
S315080066C82240826082684C79AC40224382604468E2
S315080066D89FB20126BE4024EA0604446044688A79C3
S315080066E8BA4092B222434260C2689CB2660003244A
S315080066F8B44022EA0402C260C268CC7904FA05F5F5
S315080067081543C56001330F2B16D801229A400C6829
S31508006718A243F7D104685D000322AA40D243144075
S31508006728046004680E79AE40344304600C79013C71
S31508006738E4B2012CD8D8C2E7F0BC704770470369A1
S31508006748194201D1002070470120704730B401F082
S3150800675807039B009A40C908083150F821400F25BD
S3150800676805FA03F324EA030340F8213050F82130E8
S315080067781A4340F8212030BC7047000010B4294B52
S315080067889B6803F00C03042B23D0082B24D013B1E1
S31508006798254B036001E0244B0360224CA368C3F32E
S315080067A803132249CB5CDAB20368D3404360A26874
S315080067B8C2F382228A5CD2B223FA02F28260A26803
S315080067C8C2F342328A5CD2B2D340C3605DF8044B46
S315080067D87047174B0360E0E7124B5A685B6803F08B
S315080067E83F0312F4800F12D0114AB2FBF3F20D4B95
S315080067F85B68C3F3881303FB02F30A4A5268C2F3B9
S31508006808014201325200B3FBF2F30360C5E7064AB8
S31508006818B2FBF3F2034B5B68C3F3881303FB02F37B
S31508006828EBE700BF003802400024F4000C00002003
S31508006838001BB70029B9054A136B23EA0000106341
S315080068487047024A136B18431063704700380240B2
S3150800685829B9054A536B23EA000050637047024A70
S31508006868536B1843506370470038024029B9054AE4
S31508006878136C23EA000010647047024A136C184325
S31508006888106470470038024029B9054A536C23EA50
S31508006898000050647047024A536C184350647047A6
S315080068A80038024029B9054A136923EA000010612D
S315080068B87047024A13691843106170470038024046
S315080068C829B9054A536A23EA000050627047024A02
S315080068D8536A1843506270470038024008B50121C8
S315080068E84FF40060FFF7ECFF00214FF40060FFF754
S315080068F8E7FF08BD10B40B494A6822F4FD4222F0A6
S315080069087F02037D8468234344682343C46823437A
S31508006918046823430069034313434B605DF8044B3B
S31508006928704700BF002C0140014B1860704700BF34
S31508006938A0802542014B1860704700BF002C014013
S31508006948024B186800F00300704700BF002C01408E
S3150800695810B4036809498B60CB6823F4FF6323F0F6
S315080069680703426884682243C468224300690243CD
S315080069781343CB605DF8044B704700BF002C0140F9
S31508006988014B1869C0B27047002C014082B0002339
S315080069980193034B03440193019B186802B070479F
S315080069A8142C014010B4036809494B6243688B628A
S315080069B8CA6A22F0F7028368C46823430469234332
S315080069C8406903431343CB625DF8044B704700BF25
S315080069D8002C0140014BD3F880007047002C014079
S315080069E8014BC3F880007047002C0140034B5B6BD2
S315080069F8034201D10020704701207047002C01404E
S31508006A08014B9863704700BF002C0140014B186082
S31508006A18704700BFDC00274230B585B004460D46EE
S31508006A28038A9BB223F44053CA8813430382838993
S31508006A389BB223F4B05323F00C03898828896A8902
S31508006A4801430A431343A381A38A9BB223F44073E1
S31508006A58AA891343A3826846FFF790FE204B9C42F7
S31508006A6828D003F580639C4224D0029BA28912F49D
S31508006A78004F21D103EB830303EB830329688900BD
S31508006A88B3FBF1F1174BA3FB01235809050164234E
S31508006A9800FB1313A28912F4004F16D11B013233D7
S31508006AA8104AA2FB0323C3F343132B439BB2238148
S31508006AB805B030BD039BD9E703EB830303EB8303D8
S31508006AC829684900B3FBF1F1DCE7D9003231054AF8
S31508006AD8A2FB0131C1F3421245EA0203E6E700BF09
S31508006AE8001001401F85EB5131B983899BB223F405
S31508006AF800539BB28381704783899BB243F4005342
S31508006B0883817047C1F30801818070478088C0F384
S31508006B18080070470388194201D1002070470120F0
S31508006B28704700000A4B0B4A9A6000221A60DB601D
S31508006B385A6040225A719A884FF4C86161F30C0268
S31508006B489A808022DA7041F20C0203498B5070470A
S31508006B58002200201022002000800240054B064A29
S31508006B689A60DB6000221A605A6041F210020349F3
S31508006B788B507047002F00205028002000800240C4
S31508006B882DE9F041B2B001214FF0F050FFF752FE5F
S31508006B9801214720FFF74EFE01214FF48040FFF7F9
S31508006BA873FE0120FFF732FF8E23309300258DF8F8
S31508006BB8C65002248DF8C4408DF8C7508DF8C540D4
S31508006BC85C4F30A93846FFF775FD0B220121384678
S31508006BD8FFF7BCFD0B2221463846FFF7B7FD0B2207
S31508006BE803213846FFF7B2FD0B2207213846FFF77F
S31508006BF8ADFD4FF4006330938DF8C6508DF8C44048
S31508006C088DF8C7508DF8C54007F5C05730A93846DE
S31508006C18FFF750FD0B2211463846FFF797FD32233A
S31508006C2830938DF8C6508DF8C4408DF8C7508DF846
S31508006C38C540DFF8108130A94046FFF73BFD0B2217
S31508006C4801214046FFF782FD0B2204214046FFF743
S31508006C587DFD0B2205214046FFF778FD4FF4C0431A
S31508006C6830938DF8C6508DF8C4408DF8C7508DF806
S31508006C78C54030A93846FFF71DFD0B220D213846B9
S31508006C88FFF764FD0B220E213846FFF75FFDFEF776
S31508006C98ADF8FEF7C7FAFEF7CDFA0128FBD001A82A
S31508006CA8FEF7B0F80025019508954FF400730B9385
S31508006CB80C954FF000430F932023129314951595BE
S31508006CC816954FF4006309934FF4804306931F2DD6
S31508006CD814D8ACB202212046FEF7E4F860F31F4642
S31508006CE803212046FEF7DEF860F30F06124B9E4294
S31508006CF804D0124B9E4201D00135E8E7202D0DD865
S31508006D08A9B201A8FEF72CF970B1FFF727FFFFF71C
S31508006D1809FFFEF7CDFA32B0BDE8F0814FF4A1714C
S31508006D280748FAF7CFF8EBE740F247110448FAF7AD
S31508006D38C9F8EAE70000024019162200F1C0070060
S31508006D485494000800080240064B08221A700022CC
S31508006D585A7027229A706922DA705B221A714522BC
S31508006D685A7170472C17002038B50D4B93F9033024
S31508006D78002B13DB0A4D6888C0F30D04224609491F
S31508006D88094801F06BFFEB7843F08003EB700121AB
S31508006D9841F20803054AD150204638BD002038BDBF
S31508006DA800220020102200208C1B002000800240B0
S31508006DB838B50F4B93F90330002BFADB0D4B1C88BB
S31508006DC80D4D22460D49284601F048FF084B9D609F
S31508006DD800221A60102199705A60C4F30B049C802B
S31508006DE8B022DA70012141F20403054AD15038BDB0
S31508006DF8002F0020FC1A0020502800208C1B002099
S31508006E08008002400369024A12685A6000207047E7
S31508006E18102F002010B50446D0F8E8351B699847A6
S31508006E28032384F81231002010BD08B590F81231F2
S31508006E3880F81331042380F81231D0F8E835DB6876
S31508006E489847002008BD08B5D0F8E435DB6903B1D2
S31508006E589847002008BD08B5D0F8E4351B6A984756
S31508006E68002008BD08B5D0F8E4355B6A98470020C5
S31508006E7808BD10B50446D0F8E8355B69984701237C
S31508006E8884F81531002010BD10B50446D0F8E83549
S31508006E989B699847D4F8E4355B68002120469847EB
S31508006EA8002084F8150110BD10B5044600234022B9
S31508006EB8194601F09DF8002340228021204601F05A
S31508006EC897F8012384F81231D4F8E8355B68A07876
S31508006ED89847002010BD10B582B00446694600F0F0
S31508006EE873F99DF8001001F01F03012B0FD03BB171
S31508006EF8022B11D001F08001204601F015F903E0B4
S31508006F086946204600F0D1FA002002B010BD69464D
S31508006F18204600F0EEFAF7E76946204600F006FB39
S31508006F28F2E710B5044600294CD190F81131022B26
S31508006F3805D094F81631012B3DD0002010BDD0F8A5
S31508006F483821D0F824319A4212D9D21AC0F83821F1
S31508006F58C178012906D092B2D4F82811204600F043
S31508006F68BAF8E6E7D0F828110B44C0F82831F2E752
S31508006F78D0F83C11B1FBF3F203FB12122AB98B4283
S31508006F8803D8D0F8403199420BD3D4F8E435DB68F6
S31508006F981BB194F81221032A0AD0204600F0BAF841
S31508006FA8C7E7114600F097F80023C4F84031C0E750
S31508006FB820469847F1E72046FFF724FF002384F880
S31508006FC81631BAE70A46D0F8E4355B69002BB4D01F
S31508006FD890F812110329B0D111469847ADE710B5B4
S31508006FE8044669BB90F81131032B32D1D0F8903397
S31508006FF8D0F87C23934215D99B1AC0F89033C178E8
S31508007008012909D09A4228BF1A4692B2D4F88013A1
S31508007018204600F068F81CE0D0F880131144C0F840
S315080070288013EFE7D0F8E4351B691BB190F81221F5
S31508007038032A03D0204600F05EF80AE09847F9E7E5
S315080070480A46D0F8E4359B691BB190F81211032952
S3150800705801D0002010BD11469847FAE7F8B504464E
S315080070680D4616461F4601F06DFCC4F8E475069BE6
S31508007078C4F8E835C4F8EC652946204600F06AFFE6
S31508007088D4F8E8351B689847204601F0B3FCF8BDE4
S3150800709810B50446D0F8E4351B689847D4F8E8359F
S315080070A89B689847002010BD08B5D0F8E4355B689A
S315080070B89847002008BD10B504461346C4F83C2175
S315080070C8C4F83821022280F811210A46002101F065
S315080070D808F8002010BD08B513460A46002101F035
S315080070E800F8002008BD08B513460A46002100F036
S315080070F8CAFF002008BD10B50446042380F81131DC
S3150800710800231A46194600F0ECFF204600F000FF57
S31508007118002010BD10B50446052380F81131002358
S315080071281A46194600F0AFFF204600F0F1FE002087
S3150800713810BD002302E00133DBB201300278002AD1
S31508007148F9D118467047000010B504464B88012B3C
S3150800715802D0022B0AD010BDC0F81831D0F8E43591
S315080071689B6898472046FFF7C6FF10BD8B8813F023
S31508007178FF0FF0D1026952681B0A013B042B07D896
S31508007188DFE803F0030F13171B00012363F3061246
S315080071980C4B1A60012384F816312046FFF7ABFF1B
S315080071A8D9E7022363F30612F2E7032363F3061209
S315080071B8EEE7042363F30612EAE7052363F30612E8
S315080071C8E6E700BF102F002090F8CC350B7090F832
S315080071D8CD354B7090F8CE3590F8CF2503EB0223C2
S315080071E84B8090F8D03590F8D12503EB02238B8095
S315080071F890F8D23590F8D32503EB02239BB2CB80BF
S31508007208C0F84031012380F81131704710B504469B
S31508007218802100F089FF0021204600F085FF2046DE
S3150800722800F076FE10BD30B583B005460C464A8890
S31508007238130A013B062B6ED8DFE803F00416296DFE
S315080072486D656900D0F8EC351B680DF10601807884
S315080072589847E388402B03D095F81231012B0ED1B5
S315080072680823ADF806300AE0D0F8E4359B6A0DF134
S3150800727806018078984702234370C5F8F005BDF8DB
S31508007288062012B1E388002B49D103B030BDD2B22B
S31508007298052A34D8DFE802F0030B131B232BD0F892
S315080072A8EC355B680DF1060180789847E7E7D0F872
S315080072B8EC359B680DF1060180789847DFE7D0F82A
S315080072C8EC35DB680DF1060180789847D7E7D0F8E2
S315080072D8EC351B690DF1060180789847CFE7D0F899
S315080072E8EC355B690DF1060180789847C7E7D0F851
S315080072F8EC359B690DF1060180789847BFE721466A
S31508007308FFF784FFC1E72146FFF780FFBDE721465F
S31508007318FFF77CFFB9E72146FFF778FFB5E79A42FA
S3150800732828BF1A46ADF8062001462846FFF7C3FEC9
S31508007338ABE738B504468B88E3B9CB88D3B98D78DB
S3150800734805F07F0590F81231032B0CD080F81451FC
S31508007358294600F02BFF2046FFF7CDFE35B102235C
S3150800736884F8123138BDFFF751FF38BD012384F878
S31508007378123138BD2046FFF749FF38BD10B5044617
S315080073888B78204A1370012B08D890F81221022A04
S3150800739807D0032A15D0FFF739FF10BDFFF736FFC8
S315080073A810BD5BB180F81031032280F81221194606
S315080073B8FFF76EFE2046FFF79EFE10BDFFF79BFE01
S315080073C810BD83B190F810118B4218D0FFF76CFEE8
S315080073D80C4B197884F810112046FFF759FE2046F9
S315080073E8FFF789FE10BD022280F8122180F81031B5
S315080073F81946FFF759FE2046FFF77DFE10BDFFF731
S315080074087AFE10BDF41A002008B5CB88012B08D1DE
S3150800741890F81231022B07D0032B0AD0FFF7F6FE95
S3150800742808BDFFF7F3FE08BD01220549FFF743FE2D
S3150800743808BD012200F58871FFF73DFE08BD00BFAB
S31508007448EC1A002008B590F81231023B012B0DD82A
S315080074580122084B1A60D0F8183113B10322054BDC
S315080074681A6002220349FFF726FE08BDFFF7CEFE7B
S3150800747808BD00BFE81A002010B5044690F8123176
S31508007488023B012B0ED84B88012B00D010BD0023D8
S31508007498C0F81831D0F8E4359B6898472046FFF7B6
S315080074A82AFE10BDFFF7B2FEF0E708B54B78092BA0
S315080074B81CD8DFE803F012181B151B09051B0F0C4F
S315080074C8FFF7B1FE002008BDFFF733FFFAE7FFF71D
S315080074D855FFF7E7FFF798FFF4E7FFF7B3FFF1E77C
S315080074E8FFF732FEEEE7FFF7C7FFEBE7FFF78EFE7B
S315080074F8E8E738B504460D4690F81231032B11D142
S315080075080B79012B03D9FFF781FE002038BDD0F887
S31508007518E4359B689847EB88002BF6D12046FFF799
S31508007528EAFDF2E7FFF772FEEFE7000038B5054611
S315080075380C468A88D1B26378012B25D0002B46D011
S31508007548032B1FD190F81231022B05D0032B09D033
S315080075582146FFF75BFE15E0A1B1802912D000F09D
S31508007568E3FD0FE0638823B919B1802901D000F03B
S31508007578DBFDD5F8E4359B68214628469847284612
S31508007588FFF7B9FD002038BD90F81231022B05D057
S31508007598032B0AD02146FFF739FEF3E70029F1D075
S315080075A88029EFD000F0C0FDECE76388002BE9D10D
S315080075B849B1802907D000F0D8FDD5F8E4359B688D
S315080075C82146284698472846FFF795FDDAE790F8B2
S315080075D81231022B05D0032B0AD02146FFF716FED7
S315080075E8D0E70029CED08029CCD000F09DFDC9E788
S315080075F812F0800F0FD101EB8101CB00034493F8F9
S315080076087633CBB101220E4B1A6002220C49284662
S31508007618FFF751FDB6E701F07F0101EB8101CB00C9
S31508007628034493F81E311BB10122054B1A60ECE797
S315080076380022034B1A60E8E70022014B1A60E4E7C8
S31508007648F01A0020D0B170B50D4616460446FFF765
S3150800765870FD0130400080B23080287003236B70BB
S31508007668022307E05A1CD2B20134E9540233DBB2CA
S315080076780021A95421780029F4D170BD704700006B
S31508007688C3684FF0FF325A60C3686FF080425A6188
S31508007698014BC268936170470008008030B583B013
S315080076A8054600240194032001F0A5F9EB681A6938
S315080076B8019201340E4A944217D8019A002AF2DA3E
S315080076C8019A42F001020192019A1A610023EA68B6
S315080076D8126901920133064A934203D8019A12F0B5
S315080076E8010FF4D1032001F086F9002003B030BD5C
S315080076F8400D030010B4C4786CB903339C103232B9
S3150800770800EB82008068002303E051F8042B02602E
S315080077180133A342F9D300205DF8044B704710B42F
S3150800772803329210D0F8D040002303E0206841F8CD
S31508007738040B01339342F9D308465DF8044B7047A6
S3150800774830B40023C3700123837040238380012942
S3150800775810D0E9B90023C3720C23037006234370BB
S315080077684FF4A063C3802A4CC46004F50063036120
S3150800777800231FE00123C372082303700423437000
S315080077884FF4A073C380022303724FF0A044EBE7BB
S315080077980024E9E704EB431202F51065191D00EB0E
S315080077A881018D6002F5306203F1140100EB810155
S315080077B84A60013342789342ECD304F58063436107
S315080077C804F58863C0F8CC30002309E004EB4311BC
S315080077D801F5A06103F1220200EB820291600133F0
S315080077E80578AB42F2D3002309E004EB033101F52F
S315080077F8805103F1320200EB820291600133AB42F9
S31508007808F3D304F56064C0F80C41002030BC704717
S315080078180000044038B50446037A012B16D0C2681E
S31508007828D16841F04003D360FFF738FF4FF450237F
S31508007838627A0AB14FF4E813E2689363142001F0F8
S31508007848E5F8E378012B24D0002038BD0025C26866
S31508007858936B6FF31043417A09B143F4801393632A
S31508007868E268D3686FF386136FF396536FF3514341
S315080078786FF3D343D3602046FFF710FFE378012B55
S31508007888DFD1052363F3440545F02005E3689D60C9
S31508007898D7E7E3689D68052262F3440545F02005A5
S315080078A89D60D1E7C268936843F00103936000209E
S315080078B87047C268936823F00103936000207047F5
S315080078C800B583B000230193019A42F02002019281
S315080078D8019A61F38A120192C26801991161C26814
S315080078E8126901920133074A934203D8019A12F0A2
S315080078F8200FF4D1032001F07EF8002003B05DF8CC
S3150800790804FB00BF400D030000B583B000230193B4
S31508007918019A42F010020192C26801991161C2687F
S31508007928126901920133074A934203D8019A12F061
S31508007938100FF4D1032001F05EF8002003B05DF8BB
S3150800794804FB00BF400D030008B5C268D3686FF38F
S315080079585D736FF39E73012908D009B943F0804314
S31508007968D360322001F052F8002008BD43F00053D6
S31508007978F6E7C368586900F00100704708B5FFF7CD
S31508007988F8FF10F1FF3018BF012008BDC368586911
S315080079989B69184070470269136861F3010313600D
S315080079A8704738B505460024C3689C61C3686FF0FC
S315080079B880425A61FFF764FEEB7803B9102444F055
S315080079C8804444F4701444F4605444F00C04EA689F
S315080079D8936923EA04031C439461002038BD70B5F3
S315080079E804460025D0F80C311D600269136865F352
S315080079F8CC231360C37A012B12D010212046FFF737
S31508007A085FFF2046FFF780FF236900221A61236972
S31508007A185A6123694FF0FF3199612369DA6136E0C3
S31508007A282E460321FFF7B7FFE26880235362202218
S31508007A3862F31F4563F30F05E1688D62A02161F3C0
S31508007A480F0663F31F46E368C3F804614FF490739F
S31508007A5863F30F0662F31F46E368C3F808614FF439
S31508007A68A07363F30F066FF31F46E368C3F80C6148
S31508007A78C3E74FF09041131D04EB83039868016030
S31508007A889968002008619B68FF219960013263782C
S31508007A989A4208D2131D04EB83039B681B68002BC4
S31508007AA8E7DB0021E7E700220EE04FF0904102F1FC
S31508007AB8140304EB830358680160596800200861B9
S31508007AC85B68FF219960013263789A4209D202F10C
S31508007AD8140304EB83035B681B68002BE5DB0021B2
S31508007AE8E5E72269136943F480731361E378012B88
S31508007AF804D02046FFF755FF002070BD0323402217
S31508007B0862F38A0343F4803362F3594322691363A1
S31508007B18EFE703699B68C3F34103022B04D005D832
S31508007B28012B03D0032070470120704702207047B5
S31508007B3803699B6882691168C3F34103022B0AD15A
S31508007B48032363F30A0111600269536843F48073D7
S31508007B585360002070476FF30A01F4E730B4002435
S31508007B684B78012B22D00D7805F1140200EB82021E
S31508007B7852680123AB4063F31F44136813F4004F9C
S31508007B880DD18D6865F30A03CD7865F39343897932
S31508007B9861F3995343F0805343F400431360026931
S31508007BA8D3692343D361002030BC70470D782A1D5A
S31508007BB800EB82029268AB4063F30F04DDE770B40A
S31508007BC8002215464B78012B14D00B7803F11404C0
S31508007BD800EB840464680121994061F31F456FF33B
S31508007BE8CF3222600269D36923EA0503D3610020EC
S31508007BF870BC70470E78311D00EB81018C68B34064
S31508007C0863F30F05EBE738B54B78012B25D00B78CE
S31508007C18143300EB83035B681A681C694B69002BED
S31508007C2874D18B6863F31204012363F3DC440B787D
S31508007C38143300EB83035B681C61C378012B73D08C
S31508007C48CB78012B78D042F004420B78143300EB3A
S31508007C58830043681A60002038BD0B78043300EBAC
S31508007C6883039B681A681C694B69D3B96FF31204B6
S31508007C78012363F3DC440B78043300EB83039B6826
S31508007C881C61C378012B1BD0CB78012B1FD04B69FD
S31508007C98EBB10C780123A3400469656B2B43636336
S31508007CA815E063F312048D682B44013BB3FBF5F327
S31508007CB863F3DC44CB78012BDDD163F35E74DAE732
S31508007CC80B78043300EB83039B680C695C61CB78FB
S31508007CD8012B10D042F004420B78043300EB8303DF
S31508007CE89B681A60CB78012BB5D18B8A0A78C96844
S31508007CF8FFF700FDAFE703699B6813F4807F02D19D
S31508007D0842F00052E6E742F08052E3E78D682B44DA
S31508007D18013BB3FBF5F3C3F3090363F3DC4403FB45
S31508007D2805F363F3120482E70B78143300EB830335
S31508007D385B680C695C6183E74B7913B142F00052C2
S31508007D4881E742F080527EE730B482B04B78012B47
S31508007D582ED00B78143300EB83035B681A681B690B
S31508007D6800934B69002B6DD18C689DF8003064F33D
S31508007D7806038DF800309DF80230012464F3C40325
S31508007D888DF802300B78143300EB83035B68009C8C
S31508007D981C61C378012B65D042F004420B78143372
S31508007DA800EB830043681A60002002B030BC7047B5
S31508007DB883691A681C6900944C6914BB9DF80040CD
S31508007DC86FF306048DF800409DF80240012565F317
S31508007DD8C4048DF80240009C1C61C478012C29D083
S31508007DE842F004421A60C378002BDDD14B69002B98
S31508007DF8DAD00A78012393400269516B0B4353631F
S31508007E08D2E78D68AC420ED94D619DF8004065F3FE
S31508007E1806048DF800409DF80240012565F3C40460
S31508007E288DF80240D7E79DF8005064F306058DF8EB
S31508007E380050F0E70C78043400EB8404A4680D6954
S31508007E486561CDE78C684C619DF8003064F30603DC
S31508007E588DF800309DF80230012464F3C4038DF8C8
S31508007E6802308FE70B78143300EB83035B680C69E1
S31508007E785C6191E74B78012B0AD00B78143300EB39
S31508007E8883004268116841F40013136000207047A4
S31508007E980B78043300EB830082681368002B03DB36
S31508007EA843F400131360F1E743F08043F8E74B788F
S31508007EB8012B0FD00B78143300EB83004068026857
S31508007EC86FF35552CB78023BDBB2012B08D9026017
S31508007ED8002070470B78043300EB83008068EEE7D0
S31508007EE842F08052F3E703699869DB691840000C89
S31508007EF87047143100EB81014B689A680369586921
S31508007F081040704703699869DB69184080B2704762
S31508007F1882B000230093C0238DF803304FF0000386
S31508007F28012262F3C4038DF8023018238DF8003055
S31508007F38436D009A1A61C378012B01D002B07047C5
S31508007F48436D00F2CC525A61436D1A684FF080228D
S31508007F581A60F3E738B50446FFF7F2FB012384F8FD
S31508007F681231002284F8142115E091001144CB003F
S31508007F782344012183F81D1183F81C21A3F8222123
S31508007F88002183F81F114020C3F82401C3F82811DB
S31508007F98C3F83011013260788242E6D3002214E031
S31508007FA891001144CB002344002183F8751383F804
S31508007FB87423A3F87A2383F877134025C3F87C53E8
S31508007FC8C3F88013C3F8881301328242E8D32046DF
S31508007FD8FFF76FFC2046FFF71DFC00212046FFF738
S31508007FE8B3FC2046FFF7FBFC2046FFF75BFC38BDD1
S31508007FF870B54DB2002D18DB01F07F0606EB860634
S31508008008F40004F55C740444043401F07F0121701B
S31508008018ED0F6570A260E37005B1E180022B0ED002
S315080080282146FFF79BFD002070BD01F07F0606EB91
S315080080388606F40004F58C7404440434E5E7002342
S315080080482371EDE710B54AB2002A12DB01F07F0466
S3150800805804EB8404E30003F55C730344043301F07A
S315080080687F011970D20F5A701946FFF7A8FD00202C
S3150800807810BD01F07F0404EB8404E30003F58C7358
S3150800808803440433EBE770B501F07F04A6003519FD
S31508008098E9000D4601F55C71014404312E46054494
S315080080A8C5F88023C5F888330023C5F88C3385F8C6
S315080080B8753385F87443C378012B0AD004EB840416
S315080080C8E300034493F8743343B1FFF79CFD00209B
S315080080D870BD33460344C3F88423EFE7FFF734FE3D
S315080080E8F5E770B501F07F05AE007119CC0004F507
S315080080F88C740444211D2E44F4000444012684F893
S315080081081D6184F81C51C4F82821C4F82C210022C2
S31508008118C4F83421C4F830311DB1FFF774FD0020C6
S3150800812870BDFFF711FEFAE710B54AB2002A12DB4E
S3150800813801EB8104E30003F55C730344043301246B
S315080081489C7001F07F011970D20F5A701946FFF713
S3150800815891FE002010BD01F07F0404EB8404E300BF
S3150800816803F58C7303440433E9E710B54AB2002AC9
S3150800817812DB01EB8104E30003F55C730344043363
S3150800818800249C7001F07F011970D20F5A701946A5
S31508008198FFF78DFE204610BD01F07F0404EB84042A
S315080081A8E30003F58C7303440433E9E710B40024A9
S315080081B861F30A1402691368234313605DF8044BD4
S315080081C8704708B50369596841F002025A600320E6
S315080081D800F01CFC08BD000010B50446044B1B68DB
S315080081E85B6A98474FF08043E2685361012010BDE7
S315080081F84800002038B50446C3685D6815F0040FC2
S3150800820803D1E3685D60012038BD024B1B689B6A91
S315080082189847F6E74800002010B50446837A43B124
S31508008228D0F80C316FF341036FF30003D0F80C2133
S3150800823813602269536823F001035360054B1B68D2
S315080082489B69204698474FF00043E268536101202E
S3150800825810BD00BF4800002030B583B0054600248D
S315080082688DF8074090F812318DF80730164B1B68C1
S315080082785B6998472B699A684FF40064EB685C61F8
S31508008288AB7A33B112F0010F03D095F81531012BEB
S3150800829802D0012003B030BD9DF80730DBB2032BAE
S315080082A8F7D1D5F80C21136843F001031360D5F804
S315080082B80C21136843F003031360044A136943F057
S315080082C806031361E5E700BF4800002000ED00E05B
S315080082D810B50446044B1B68DB6898470823E26810
S315080082E85361012010BD00BF4800002010B50446A0
S315080082F8044B1B68DB6998474FF48013E26853619F
S31508008308012010BD4800002010B50446044B1B6820
S315080083181B6A98474FF40013E2685361012010BDA1
S315080083284800002003691A695B6BCB40DB01DBB2A6
S315080083381343043100EB810082689068184070473F
S315080083482DE9F0410746FFF7CEFD0446002520E053
S3150800835805F1140307EB83035B681969AA002A4425
S31508008368D3003B44D3F87C23C1F31201521AC3F84D
S315080083788C2327E016F0020F06D0022605F114030F
S3150800838807EB83035B689E6016F0080F2DD101354D
S315080083986408002C36D014F0010FF8D05FFA85F877
S315080083A841463846FFF7A5FD064610F0010FE1D00D
S315080083B8012605F1140307EB83035B689E60FB78C7
S315080083C8B342C5D0114B1B681B68414638469847C7
S315080083D8FB78012BCED1002DCCD197F81131052B7E
S315080083E8C8D13846FFF794FDC4E7084B1B689B6855
S315080083F838469847082605F1140307EB83035B6894
S315080084089E60C4E70120BDE8F08100BF480000204F
S315080084182DE9F04107460D468A000A44D30003446D
S31508008428D3F83021D3F83411521AD3F824319A42A2
S3150800843800D8134603F103084FEA98082B1D07EBE3
S3150800844883039B689B691DE006F103084FEA9808B1
S31508008458AB002B44DC003C44B3B2EAB2D4F828118A
S315080084683846FFF747F9D4F828313344C4F8283191
S31508008478D4F834311E44C4F834612B1D07EB830342
S315080084889B689B699BB2984515D2AB002B44DA00CA
S315080084983A44D2F83411D2F8303199420BD253B152
S315080084A85B1A05EB8501CA003A44D2F82461B3423F
S315080084B8CAD81E46C8E70120BDE8F0812DE9F04173
S315080084C80746FFF71FFD0446002624E0012303FAA2
S315080084D806F039694A6B22EA00024A631D46321DCC
S315080084E807EB8202926893602C4B1B685B684146CF
S315080084F838469847FB78AB421CD1DEB997F8113154
S31508008508042B17D13846FFF703FD13E015F0800F43
S3150800851835D101366408002C3CD014F0010FF8D088
S315080085285FFA86F841463846FFF7FCFE054610F01E
S31508008538010FCBD115F0080F05D00825331D07EB19
S3150800854883039B689D6015F0100F05D01025331D11
S3150800855807EB83039B689D6015F0400F05D04025FF
S31508008568331D07EB83039B689D6015F0020FCDD07A
S315080085780225331D07EB83039B689D60C6E73146D2
S315080085883846FFF745FF8025331D07EB83039B68AD
S315080085989D60BEE70120BDE8F08100BF48000020C5
S315080085A82DE9F0410446C268936923F010039361E4
S315080085B8C3681D6A05F00F06C5F34343022B09D0A5
S315080085C8062B23D0E268936943F0100393610120D0
S315080085D8BDE8F08147F6F0732B42F3D0C5F30A15C8
S315080085E84FEA860808EB0603DF0007442A46D7F849
S315080085F88013FFF794F8D7F880332B44C7F88033ED
S31508008608D7F88C331D44C7F88C53DBE7082200F2E9
S31508008618CC51FFF784F8C5F30A15B3009919CA00AF
S315080086282244D2F88C331D44C2F88C53CAE700009A
S315080086382DE9F84304460025A8462F462E46026922
S31508008648536823F0010353602946FFF739F92B4687
S315080086580CE01A1D04EB82029268FF21916003F16F
S31508008668140204EB820252689160013362789342DD
S31508008678EFD323694FF0FF329A614FF0010969F386
S315080086880F0569F31F452369DD6148F00B0823695F
S31508008698C3F8148047F00B0723691F61226913681A
S315080086A86FF30A1313602046FFF732FC46F4805628
S315080086B8E3685E61034B1B681B6920469847484672
S315080086C8BDE8F8834800002038B50446FFF730FAB5
S315080086D8E368DD682046FFF71CFA03280ED0012355
S315080086E8A3704023A380052363F38D25E368DD6023
S315080086F84FF40053E2685361012038BD0023A37084
S315080087084FF40073A380092363F38D25EEE72DE95B
S31508008718F8430546FFF732F918B900242046BDE89C
S31508008728F8832846FFF732F9044606460028F5D0A6
S31508008738C0F3074818F0080F33D1002418F0040FBF
S3150800874834D1F7B217F0020F02D00223EA68536150
S31508008758C6F307635FFA83F913F0800F2BD1C6F3C4
S31508008768072616F0080F2BD117F0080F2DD117F08A
S31508008778100F2FD116F0100F31D116F0200F33D164
S3150800878818F0100F35D118F0200F37D119F0400F0F
S3150800879839D117F0040FC1D02846FFF72BFD04433B
S315080087A8BCE72846FFF7CCFD0446C7E72846FFF787
S315080087B885FE0443C5E72846FFF72EFD0443CEE7A2
S315080087C82846FFF749FD0443CEE72846FFF780FD0C
S315080087D80443CCE72846FFF7E3FE0443CAE72846DE
S315080087E8FFF726FF0443C8E72846FFF76DFF04434B
S315080087F8C6E72846FFF77AFD0443C4E72846FFF785
S3150800880883FD0443C2E72846FFF7E6FC0443C0E7AE
S31508008818F0B583B0FDF778FE01210846FEF70AF899
S315080088280124009400268DF804608DF80760022557
S315080088388DF8055069462848FDF73CFF2146202053
S31508008848FEF722F821460420FDF7F4FF234F0822F5
S3150800885806213846FDF77AFF082207213846FDF72C
S3150800886875FF8DF806608DF807408DF8045040238B
S3150800887800938DF8055069463846FDF71BFF8DF8B5
S3150800888804508023009369463846FDF713FF2146AE
S315080088982846FDF7CFFFA7F5806709220521384640
S315080088A8FDF754FF092206213846FDF74FFF6023D6
S315080088B800938DF804508DF805508DF806608DF8EC
S315080088C8074069463846FDF7F5FE21464FF0C06071
S315080088D8FDF7CCFF03B0F0BD0000024000080240D7
S315080088E808B5FFF795FFF8F725FBF8F733FBFCE71C
S315080088F8DFF834D0002103E00C4B5B5843500431B1
S315080089080B480C4B42189A42F6D30B4A02E000234E
S3150800891842F8043B094B9A42F9D3FDF7F5FD00F0F6
S3150800892859F9FFF7DDFF704700000220D0950008C7
S3150800893800000020B8020020000300205430002060
S31508008948FEE70000F0B583B001210846FDF772FF7F
S315080089584FF4C853009303278DF8057002238DF842
S31508008968043000268DF806608DF80760204C6946A5
S315080089782046FDF79FFE0A2208212046FDF7E6FE57
S315080089880A220B212046FDF7E1FE0A220C21204681
S31508008998FDF7DCFE4FF4007300938DF805708DF82B
S315080089A8046001258DF806508DF80760694620464B
S315080089B8FDF780FE4FF4806300938DF806508DF816
S315080089C807508DF8057069462046FDF773FE0A229A
S315080089D811462046FDF7BAFE29464FF48040FDF7B2
S315080089E853FF29468020FDF733FF03B0F0BD00BFCB
S315080089F800000240704704E000BF01331B2BFBD977
S31508008A081046421E08B10023F8E7704708B54FF428
S31508008A187A7303FB00F0FFF7EEFF08BD20230B80EF
S31508008A28004870477800002008B590F81231032BE3
S31508008A3801D0002008BDF8F7E3F9FAE708B5F8F712
S31508008A48DFF9002008BD08B50846F8F70DFA002032
S31508008A5808BD000008B50B7813F0600F06D14B78EF
S31508008A680A2B14D00B2B17D0062B01D0002008BDD3
S31508008A784B881B0A212B04D00B491722FEF71BFB30
S31508008A88F4E7CA88172A28BF17220849F6E70122F1
S31508008A980749FEF710FBE9E78B7813B9044A136010
S31508008AA8E4E7FEF7B3FBE1E7810000208A0000202F
S31508008AB8F81A002010B504468121FFF7C3FA0121E8
S31508008AC82046FFF7BFFA002010BD000010B504467F
S31508008AD8022340228121FFF78BFA02234022012133
S31508008AE82046FFF785FA4023034A01212046FFF767
S31508008AF8CAFA002010BD00BF14300020004870478D
S31508008B081430002012230B80004870479800002074
S31508008B1804230B8000487047AC00002010B5044CAD
S31508008B280A4621460348FEF78DFD204610BD00BFBC
S31508008B38142F00209894000810B5044C0A462146BC
S31508008B480348FEF77FFD204610BD00BF142F0020FE
S31508008B588894000810B5044C0A4621460348FEF7CF
S31508008B6871FD204610BD00BF142F0020AC940008E4
S31508008B7810B5044C0A4621460348FEF763FD20460D
S31508008B8810BD00BF142F00206894000810B5044CC7
S31508008B980A4621460348FEF755FD204610BD00BF84
S31508008BA8142F00207094000870477047704708B55E
S31508008BB8FCF77FF808BD08B5FCF77CF808BD08B5CA
S31508008BC80120FCF775F808BD08B50020FCF770F811
S31508008BD808BD000070B50D4E0D4CA41BA410002549
S31508008BE8A54209D10B4E0C4C00F058F8A41BA4104A
S31508008BF80025A54205D170BD56F825309847013598
S31508008C08EEE756F8253098470135F2E7C895000883
S31508008C18C8950008C8950008CC950008044B054A6D
S31508008C281B681B6A002B08BF1346D3F8EC0070476D
S31508008C3854020020E800002082B001B901A942B117
S31508008C484BB113780B601278101C18BF012002B0BC
S31508008C5870471046FBE76FF00100F8E710B5431EAA
S31508008C680A44914200D110BD11F8014B03F8014F8F
S31508008C78F7E702440346934200D1704703F8011BFD
S31508008C88F9E749B1FF2A85BF8A2303600A704FF0BE
S31508008C98FF3098BF0120704708467047F8B500BFEF
S31508008CA8F8BC08BC9E467047F8B500BFF8BC08BCB7
S30908008CB89E4670470F
S31508008CBC2E2E2F2E2E2F2E2E2F2E2E2F536F7572C5
S31508008CCC63652F41524D434D345F53544D333246F1
S31508008CDC342F63616E2E6300050206020603070332
S31508008CEC0803090309040A040B040C040C050D05F6
S31508008CFC0E050F050F0610061007100800C0000811
S31508008D0C00400000030000000000010800000100FC
S31508008D1C0400000000000208000002000500000024
S31508008D2C0000040800000200060000000000060807
S31508008D3C00000200070000000000080800000200FE
S31508008D4C0800000000000A080000020009000000E4
S31508008D5C00000C08000002000A00000000000E08C3
S31508008D6C000002000B0000000000080010001800AC
S31508008D7C20002800300038004000480050005800F9
S31508008D8C8000880090009800A000A800B000B800E9
S31508008D9CC000C800D000D8002E2E2F2E2E2F2E2E17
S31508008DAC2F2E2E2F536F757263652F41524D434DDF
S31508008DBC345F53544D333246342F756172742E63B7
S31508008DCC000000002E2E2F2E2E2F2E2E2F2E2E2F5D
S31508008DDC536F757263652F41524D434D345F53542F
S31508008DEC4D333246342F7573622E6300303A0000C9
S31508008DFC2E2E2F2E2E2F2E2E2F2E2E2F536F757284
S31508008E0C63652F66696C652E630000004669726D92
S31508008E1C7761726520757064617465207265717509
S31508008E2C6573742064657465637465640A0D000063
S31508008E3C4F70656E696E67206669726D77617265CB
S31508008E4C2066696C6520666F722072656164696E4E
S31508008E5C672E2E2E000000004552524F520A0D0066
S31508008E6C4F4B0A0D000000005374617274696E67EB
S31508008E7C207468652070726F6772616D6D696E67B4
S31508008E8C2073657175656E63650A0D0050617273A2
S31508008E9C696E67206669726D776172652066696CA2
S31508008EAC6520746F206465746563742065726173DC
S31508008EBC6520626C6F636B732E2E2E004572617380
S31508008ECC696E67200000000020627974657320665D
S31508008EDC726F6D206D656D6F7279206174203078B4
S31508008EEC0000000052656164696E67206C696E65E6
S31508008EFC2066726F6D2066696C652E2E2E45525251
S31508008F0C4F520A0D00000000496E76616C696420A8
S31508008F1C636865636B73756D20666F756E642E2E4C
S31508008F2C2E4552524F520A0D0000000050726F67C0
S31508008F3C72616D6D696E672000000000206279749D
S31508008F4C657320746F206D656D6F7279206174205E
S31508008F5C3078000057726974696E672070726F6793
S31508008F6C72616D20636865636B73756D2E2E2E00AA
S31508008F7C436C6F73696E67206669726D776172658B
S31508008F8C2066696C650A0D004669726D77617265B3
S31508008F9C2075706461746520737563636573736695
S31508008FAC756C6C7920636F6D706C657465640A0DED
S31508008FBC00000000809A45418E418F804545454901
S31508008FCC49498E8F9092924F994F555559999A9B1C
S31508008FDC9C9D9E9F41494F55A5A5A6A7A8A9AAAB96
S31508008FECACADAEAFB0B1B2B3B4B5B6B7B8B9BABB2F
S31508008FFCBCBDBEBFC0C1C2C3C4C5C6C7C8C9CACB1F
S3150800900CCCCDCECFD0D1D2D3D4D5D6D7D8D9DADB0E
S3150800901CDCDDDEDFE0E1E2E3E4E5E6E7E8E9EAEBFE
S3150800902CECEDEEEFF0F1F2F3F4F5F6F7F8F9FAFBEE
S3150800903CFCFDFEFF01030507090E10121416181C79
S3150800904C1E000000222A3A3C3E3F7C7F00000000AE
S3150800905C2B2C3B3D5B5D0000C700FC00E900E200E1
S3150800906CE400E000E500E700EA00EB00E800EF00AA
S3150800907CEE00EC00C400C500C900E600C600F4000A
S3150800908CF600F200FB00F900FF00D600DC00A20097
S3150800909CA300A500A7209201E100ED00F300FA0059
S315080090ACF100D100AA00BA00BF001023AC00BD0025
S315080090BCBC00A100AB00BB00912592259325022587
S315080090CC24256125622556255525632551255725C1
S315080090DC5D255C255B251025142534252C251C259A
S315080090EC00253C255E255F255A25542569256625C8
S315080090FC602550256C256725682564256525592521
S3150800910C5825522553256B256A2518250C2588259F
S3150800911C84258C2590258025B103DF009303C00395
S3150800912CA303C303B500C403A6039803A903B40396
S3150800913C1E22C603B50329226122B10065226422C8
S3150800914C20232123F7004822B0001922B7001A223F
S3150800915C7F20B200A025A00061001A03E0001703C7
S3150800916CF8000703FF000100780100013001320105
S3150800917C0601390110014A012E0179010601800107
S3150800918C4D0043028101820182018401840186011A
S3150800919C8701870189018A018B018B018D018E015B
S315080091AC8F0190019101910193019401F6019601A9
S315080091BC9701980198013D029B019C019D01200293
S315080091CC9F01A001A001A201A201A401A401A6016C
S315080091DCA701A701A901AA01AB01AC01AC01AE011B
S315080091ECAF01AF01B101B201B301B301B501B501CC
S315080091FCB701B801B801BA01BB01BC01BC01BE017B
S3150800920CF701C001C101C201C301C401C501C401F2
S3150800921CC701C801C701CA01CB01CA01CD0110019A
S3150800922CDD0101008E01DE011201F3010300F101DB
S3150800923CF401F401F8012801220212013A0209008C
S3150800924C652C3B023B023D02662C3F024002410262
S3150800925C410246020A015302400081018601550269
S3150800926C89018A0158028F015A0290015C025D023B
S3150800927C5E025F0293016102620294016402650256
S3150800928C66026702970196016A02622C6C026D02ED
S3150800929C6E029C01700271029D01730274029F0199
S315080092AC76027702780279027A027B027C02642CB7
S315080092BC7E027F02A60181028202A901840285022E
S315080092CC86028702AE014402B101B20145028D0243
S315080092DC8E028F0290029102B7017B030300FD03F5
S315080092ECFE03FF03AC0304008603880389038A0381
S315080092FCB1031103C2030200A303A303C4030803A7
S3150800930CCC0303008C038E038F03D8031801F203D6
S3150800931C0A00F903F303F403F503F603F703F7035B
S3150800932CF903FA03FA033004200350041007600407
S3150800933C22018A043601C1040E01CF040100C004BF
S3150800934CD004440161052604000000007D1D0100BF
S3150800935C632C001E9601A01E5A01001F0806101F3A
S3150800936C0606201F0806301F0806401F0606511F52
S3150800937C0700591F521F5B1F541F5D1F561F5F1F87
S3150800938C601F0806701F0E00BA1FBB1FC81FC91F17
S3150800939CCA1FCB1FDA1FDB1FF81FF91FEA1FEB1FAB
S315080093ACFA1FFB1F801F0806901F0806A01F080639
S315080093BCB01F0400B81FB91FB21FBC1FCC1F010079
S315080093CCC31FD01F0206E01F0206E51F0100EC1F93
S315080093DCF21F0100FC1F4E210100322170211002E0
S315080093EC842101008321D0241A05302C2F04602CEB
S315080093FC0201672C0601752C0201802C6401002DD4
S3150800940C260841FF1A030000FFFFFFFFFFFF0000BD
S3150800941C4F70656E424C54002F626F6F746C6F6799
S3150800942C2E747874000000002F64656D6F70726F6F
S3150800943C675F6F6C696D65785F73746D333265340D
S3150800944C30372E73726563002E2E2F6C69622F755A
S3150800945C69702F6E65746465762E63004465666163
S3150800946C756C740057696E5553422042756C6B20A7
S3150800947C496E746572666163650000004F70656EAF
S3150800948C424C5420557365720000000057696E559E
S3150800949C53422042756C6B204465766963650000FF
S315080094AC303030303030303030353043000000004A
S315080094BC4300504F534958002E00002020202020EE
S315080094CC202020202828282828202020202020205A
S315080094DC202020202020202020202088101010104A
S315080094EC101010101010101010101004040404049E
S315080094FC04040404041010101010101041414141CA
S3150800950C41410101010101010101010101010101B1
S3150800951C01010101010110101010101042424242C3
S3150800952C4242020202020202020202020202020281
S3150800953C02020202020210101010200000000000A5
S3150800954C0000000000000000000000000000000001
S3150800955C00000000000000000000000000000000F1
S3150800956C00000000000000000000000000000000E1
S3150800957C00000000000000000000000000000000D1
S3150800958C00000000000000000000000000000000C1
S3150800959C00000000000000000000000000000000B1
S315080095AC00000000000000000000000000000000A1
S311080095BC00000000000000000000000095
S309080095C8AD010008DB
S309080095CC89010008FB
S315080095D00400000001000000010000000000000077
S315080095E0010203040102030406070809E76F0008DD
S315080095F02B6F0008DF6E00084F6E0008B16E00087A
S31508009600336E00081D6E00085F6E00086D6E000858
S315080096107B6E0008916E00081C000020D58A0008A1
S31508009620BD8A00085D8A00080000000000000000EE
S31508009630458A00084F8A0008318A000800000000A1
S3150800964000000000258A000809022000010100C068
S31508009650320904000002FF000000070581024000ED
S31508009660FF070501024000FF12011001000000403B
S31508009670501DAC6000010102030100000403090447
S315080096800D8B0008198B0008418B0008258B0008F4
S315080096905D8B0008798B0008958B0008B18B000854
S315080096A0B38B0008B58B0008B78B0008BF8B000882
S315080096B0C78B0008D18B000843000000000000009B
S315080096C0000000000000000000000000000000008C
S315080096D00000000000000000430000000000000039
S315080096E0000000000000000000000000000000006C
S315080096F00000000000000000430000000000000019
S31508009700000000000000000000000000000000004B
S3150800971000000000000000004300000000000000F8
S31508009720000000000000000000000000000000002B
S3150800973000000000000000004300000000000000D8
S31508009740000000000000000000000000000000000B
S3150800975000000000000000004300000000000000B8
S3150800976000000000000000000000000000000000EB
S315080097700000000000000000430000000000000098
S3150800978000000000000000000000000000000000CB
S3150800979000000000000000008B8C0008418C0008C7
S315080097A000000000C6940008C4940008C594000888
S315080097B0C5940008C5940008C5940008C594000817
S315080097C0C5940008C5940008C5940008C594000807
S315080097D0FFFFFFFFFFFFFFFFFFFFFFFFFFFF000089
S315080097E00100415343494900000000000000000001
S315080097F0000000000000000000000000000000005B
S3150800980000004153434949000000000000000000E1
S31508009810000000000000000000000000000000003A
S3150800982000000000580200200000000000000000B0
S31508009830000000000000000000000000000000001A
S31508009840000000000000000000000000000000000A
S3150800985000000000000000000000000000000000FA
S3150800986000000000000000000000000000000000EA
S3150800987000000000000000000000000000000000DA
S30D080098800000000000000000D2
S705080088F971
